:020000040800F2
:10000000A80E002079020008092D00086F150008CD
:10001000F92B0008A50900087F3C0008000000003B
:10002000000000000000000000000000C1330008D4
:10003000990A000800000000A12D00088D3A000870
:10004000930200089302000893020008930200083C
:10005000930200089302000893020008930200082C
:10006000930200089302000893020008930200081C
:100070009302000893020008050A00089302000892
:1000800093020008250A0008930200089302000862
:1000900093020008930200089302000893020008EC
:1000A00093020008930200089302000893020008DC
:1000B00093020008753B00089302000893020008B1
:1000C00093020008930200089302000893020008BC
:1000D00093020008713C0008733C0008773C00085C
:1000E000930200089302000893020008930200089C
:1000F000930200089302000893020008930200088C
:10010000930200089302000893020008930200087B
:100110009302000893020008930200086D3C000857
:10012000450A0008750A00089302000893020008B7
:10013000930200089302000893020008930200084B
:10014000930200089302000893020008930200083B
:1001500093020008790A0008930200087B3C00081B
:10016000930200089302000893020008930200081B
:1001700093020008930200089302000800000000A8
:10018000930200089302000800F002F800F064F8FF
:100190000AA090E8000C82448344AAF10107DA45E2
:1001A00001D100F059F8AFF2090EBAE80F0013F0D0
:1001B000010F18BFFB1A43F001031847C478000071
:1001C000E47800000A444FF0000C10F8013B13F0F3
:1001D000070408BF10F8014B1D1108BF10F8015BA0
:1001E000641E05D010F8016B641E01F8016BF9D193
:1001F00013F0080F1EBF10F8014BAD1C0C1B09D1EA
:100200006D1E58BF01F801CBFAD505E014F8016B5B
:1002100001F8016B6D1EF9D59142D6D370470000ED
:100220000023002400250026103A28BF78C1FBD8FF
:10023000520728BF30C148BF0B607047632900F0E8
:100240003E82732900F04382002070471FB507F0FB
:10025000ADFA1FBD10B510BD00F078FA1146FFF7DA
:10026000F5FF05F03FFF00F096FA03B4FFF7F2FF49
:1002700003BC00F097FA000009488047094800478E
:10028000FEE7FEE7FEE7FEE7FEE7FEE7FEE7FEE746
:10029000FEE7FEE704480549054A064B70470000A3
:1002A000653B000889010008A8080020A80E00206E
:1002B000A80A0020A80A002053EA020C00F0698076
:1002C0002DE9F04B4FF00006002B1FBFB3FA83F56A
:1002D00003FA05F424FA05F65E4012BF1643B2FA9B
:1002E00082F502FA05F4C5F120051EBF22FA05FCCD
:1002F00044EA0C04203556EA044C4FEA144418BF73
:10030000641C4FF000084FF00009904271EB030CA1
:1003100039D3002919BFB1FA81F701FA07F6B0FA0B
:1003200080F700FA07F6C7F120071EBF20FA07FC86
:1003300046EA0C062037B6FBF4FCA7EB0507103F96
:1003400007F01F0BCBF120060CFA0BFB2CFA06F67C
:1003500044BFB3460026202FA4BF5E464FF0000BDB
:100360005BEA060C08BF4FF0010B19EB0B09ABFB66
:10037000027C48EB0608C01B06FB02CC0BFB03CC3F
:1003800071EB0C01C1E70B46024641464846BDE809
:10039000F08B13B54FF000004FF00001AFF3008079
:1003A000BDE81C40704700000FB41CB50C0007AA44
:1003B000009001D02044401E074B7B4469460190C9
:1003C000069800F052F9002C03D06946002000F096
:1003D0005FF91CBC5DF814FBDD0200002DE9F04163
:1003E0000E460446002020622046E168884730B36C
:1003F000252805D0D4E901219047206A401CF2E766
:10040000E168204600278847050018D0A5F1410083
:10041000192802D820354FF4006732462946204675
:100420002760FFF70BFF40B1012804D0F61D26F02E
:1004300007060836D8E7361DD6E72846DAE7206AE9
:10044000BDE8F08170B50C460546012A05D0287834
:10045000800600D5EA69002302E0012305E05B1C69
:10046000934202D2E05C0028F9D1A869E618C01ACC
:10047000A861286A184428622846AFF3008004E087
:10048000D5E9012114F8010B9047B442F8D328466E
:10049000AFF3008070BD10B5431C02E010F8011BE3
:1004A00071B18107FAD14FF0013202C88C1A8C4326
:1004B00014EAC211F9D0C01A0A0603D0C01E10BD3A
:1004C000C01A10BD0A0401D0801E10BD0902FCD064
:1004D000401E10BD40EA010370B59B072ED14FF0BE
:1004E0000136042A2AD308C810C99D1B9D43121F38
:1004F00015EAC61517D0D8B2E1B2401A50EA056124
:1005000010D198B2A1B2401A50EA05410AD123F0A5
:100510007F4024F07F41401A50EA052102D1180E95
:10052000A0EB146070BDA342DBD018BA21BA884298
:1005300001D9012070BD4FF0FF3070BD0AB9002015
:1005400070BD10F8013B11F8014B63B1A3420AD111
:10055000521E08D010F8013B11F8014B1BB1A34209
:1005600001D1521EEDD1181B70BD032A40F230801C
:1005700010F0030C00F0158011F8013BBCF1020FE4
:10058000624498BF11F801CB00F8013B38BF11F865
:10059000013BA2F1040298BF00F801CB38BF00F87C
:1005A000013B11F0030300F09680083AC0F0088088
:1005B00051F8043B083A51F804CBA0E80810F5E7DD
:1005C000121D5CBF51F8043B40F8043BAFF30080C0
:1005D000D20724BF11F8013B11F801CB48BF11F835
:1005E000012B24BF00F8013B00F801CB48BF00F805
:1005F000012B70474FF0000200B513469446964613
:10060000203922BFA0E80C50A0E80C50B1F1200125
:10061000BFF4F7AF090728BFA0E80C5048BF0CC0D3
:100620005DF804EB890028BF40F8042B08BF704731
:1006300048BF20F8022B11F0804F18BF00F8012BA3
:10064000704770477047704710B500F077F8006842
:1006500010BD10B5044600F071F8046010BD000034
:1006600001694A1C02610878704700B58FB0CDE976
:1006700001310021059105497944CDE90310114666
:100680006846FFF7ABFE0FB000BD0000E5FFFFFFBF
:100690000A6802F8010B0A607047D1E900239A4208
:1006A00002D2531C0B601070704710B5436913B130
:1006B000AFF3008001E0FFF7C5FE012010BD127806
:1006C00000F124010A7000224A700122EDE711684E
:1006D0004FF0FF32E9E710B5203AC0F00B80B1E8E7
:1006E0001850203AA0E81850B1E81850A0E8185067
:1006F000BFF4F5AF5FEA027C24BFB1E81850A0E870
:10070000185044BF18C918C0BDE810405FEA827C89
:1007100024BF51F8043B40F8043B08BF7047D207A0
:1007200028BF31F8023B48BF11F8012B28BF20F841
:10073000023B48BF00F8012B70470000004870479B
:100740004408002000487047440800207546FFF721
:10075000F9FFAE4605006946534620F0070085467E
:1007600018B020B5FFF796FDBDE820404FF0000619
:100770004FF000074FF000084FF0000B21F0070189
:10078000AC46ACE8C009ACE8C009ACE8C009ACE8CC
:10079000C0098D4670470446AFF300802046FFF73E
:1007A00064FD000001491820ABBEFEE726000200F0
:1007B000704700002DE9F04107462DED028B82B015
:1007C0000025474EDFF81C81474C0DE02168491C8D
:1007D00021603068814207DB256094ED040B02B094
:1007E000BDEC028BBDE8F0810121404601F039F9F2
:1007F0000028EBD1082F2CD2DFE807F004090E13F4
:10080000181D22270821012000F076F821E0182188
:10081000012000F071F81CE02821012000F06CF8A4
:1008200017E03821012000F067F812E0482101208C
:1008300000F062F80DE05821012000F05DF808E0BA
:100840006821012000F058F803E07821012000F031
:1008500053F8FC20019001231A4601A9234800F017
:10086000ADFC019501231A4601A9204800F0A6FC21
:100870000120019001231A4601A91C4800F09EFCAA
:10088000012303226946194800F0ECFB9DF80000A3
:100890009DF80110000440EA01209DF80210084371
:1008A0006060A0609FED128B01020ED5C043C0F3C3
:1008B0001600401C4042A06006F0CBFB53EC182B06
:1008C00006F07EFCC4E9040107E006F0C2FB53EC2D
:1008D000182B06F075FCC4E9040194ED040B7EE7C7
:1008E00018000020000C024000010020300200200F
:1008F00085F90F270088433F2DE9F34182B0074671
:100900000025164C164EDFF85C8008E02168491C73
:1009100021603068814202DB2560BDE8FF81012152
:10092000404601F09EF80028F0D107F00F0040F09B
:100930005000019001231A4601A90B4800F03EFC2B
:10094000019501231A4601A9074800F037FC01234D
:100950001A4603A9044800F031FCDEE7000100203C
:1009600018000020000C02403002002010B50220C8
:100970000B49886106210020FFF7BEFF08210120F6
:10098000FFF7BAFF00210220FFF7B6FFF021032096
:10099000FFF7B2FF0021BDE810400420FFF7ACBF15
:1009A000000C0240FEE7000070B512484FF4001240
:1009B00053100578104894101049092D07D2DFE82C
:1009C00005F0060507090B0E10121400826170BDB8
:1009D000836170BD846170BD0421816170BD8A61D5
:1009E00070BD8B6170BD8C6170BD802004498861D1
:1009F00070BD0000240100200010024000040240ED
:100A0000000C024006480168C1F3C061002905D00E
:100A10004FF000618160032100F0B0BE704700001C
:100A20000060024006484168C1F34051002905D0EA
:100A30004FF40011C160062100F0A0BE7047000015
:100A40000060024009480168C1F34011002902D04A
:100A5000074A01211170202181600168C1F3C001A2
:100A6000002901D008218160704700000064024025
:100A70003C0000207047000006484168C1F3405127
:100A8000002905D04FF40011C160062100F076BEA8
:100A90007047000000640240704772B6FEE7000035
:100AA000024931F8100080B270470000DE000020DB
:100AB000024931F8100080B270470000AC000020FD
:100AC00010B51038C21700EB5272084CD310E35C1B
:100AD00022F00702821A012404FA02F0184201D01F
:100AE0000C7010BD0020087010BD0000A800002090
:100AF00010B5084A02EBD002127800F00704012377
:100B000003FA04F0104201D00B7010BD00200870F1
:100B100010BD0000AA0000202DE9F0412A4C00265B
:100B200026610221A22002F0A5F904F11005274F49
:100B3000A878697800EB0120217827F81100266158
:100B40000221A42002F096F9A878697800EB012030
:100B5000217807EB4101088226610221A62002F0DC
:100B600089F9A878697800EB0120217807EB410129
:100B7000088426610221A82002F07CF9A87869780F
:100B800000EB0120217807EB410108862661022154
:100B9000AA2002F06FF9A878697800EB012021788B
:100BA00007EB4101A1F8400026610221AC2002F0D0
:100BB00061F9A878697800EB0120217807EB410101
:100BC000A1F85000BDE8F08124010020DC060020DF
:100BD0002DE9F84F0022DFF89C914FF00108032720
:100BE0004FF00F0C09F1040AA9F1040B08FA02F501
:100BF0000B682B40AB426ED10C7904F00304012C3E
:100C000001D0022C15D18668540007FA04FE26EAAA
:100C10000E06D1F80CE00EFA04FE4EEA060EC0F8FD
:100C200008E04468AC430D79C5F3001595402543B1
:100C300045600C79E443A40708D0C568540007FA5E
:100C400004F6B5438E68A6402E43C6600C7904F0C6
:100C50000304022C11D1D40800EB8406356A540732
:100C6000E40E0CFA04FE25EA0E05D1F810E00EFAA7
:100C700004FE4EEA050EC6F820E00568540007FAA7
:100C800004F6B5430E7906F00306A6402E4306602F
:100C90004C6814F4403F67D0374C256845F48045D4
:100CA0002560246804F480440094344C22F0030549
:100CB0002E19D6F8085894074FEA147E0CFA0EF451
:100CC000A5432F4CA04201D1002424E02D4CA0428A
:100CD00002D101241FE047E02B4CA04201D10224A5
:100CE00019E02A4CA04201D1032414E0284CA04270
:100CF00001D104240FE0274CA04201D105240AE0D1
:100D0000254CA04201D1062405E0244CA04201D18B
:100D1000072400E0082404FA0EF42C43C6F808481F
:100D2000D9F800409C434D68ED0200D51C43C9F83A
:100D30000040DAF800409C434D68AD0200D51C43EA
:100D4000CAF80040DBF800409C434D68AD0300D575
:100D50001C43CBF80040074D083D2C689C434E686F
:100D6000F60300D51C432C60521C102AFFF43EAF42
:100D7000BDE8F88F083C0140443802400030014093
:100D8000000002400004024000080240000C024043
:100D9000001002400014024000180240001C0240F3
:100DA0000148806870470000980000200248816870
:100DB00002781144816070479800002010B50B48FC
:100DC000016841F400710160016841F480610160D3
:100DD000016841F480710160032000F065F8002093
:100DE00000F006F800F026F8002010BD003C02409C
:100DF00070B504460D4D4FF47A712878B1FBF0F0D0
:100E00000B490968B1FBF0F000F09DFB08B101202F
:100E100070BD102C07D200222146501E00F024F88D
:100E20006C60002070BD012070BD000098000020A3
:100E3000A400002082B00B48016841F480410160A9
:100E4000006800F4804001900648001F016841F0EE
:100E500080510160006800F080500190052002B0D0
:100E600000F022B844380240F0B40D460D4B1B6828
:100E7000C3F30223C3F10704042C00D90424191D71
:100E8000072901D2002300E0DB1E012606FA04F147
:100E9000491E294099409E40761E16403143F0BCC1
:100EA00003F058B90CED00E000F00701054A1068A6
:100EB0004FF6FF03184040EA012003490843106041
:100EC000704700000CED00E00000FA0570B5044624
:100ED000002C09D0606A002540B125616561A562DA
:100EE00094F8510040B10CE0012070BD6068B0F58D
:100EF000827FF4D0E561F2E784F85050204600F09C
:100F000045F8022084F851002068016821F0400172
:100F10000160A088218900F4827001F40441084333
:100F2000A18901F400610843217C01F0020108431A
:100F3000217D01F001010843218B01F40071084378
:100F4000217F01F03801084394F8201001F080015E
:100F50000843218D01F40051084321680860A0690D
:100F6000042101EA104094F8241001F01001084314
:100F7000216848602068C16921F40061C16165652C
:100F8000012084F85100002070BD0000F0B587B04A
:100F90000446142102A8FFF72DFB2D4B22680024E4
:100FA0002C49022503262C489A421DD1294A143285
:100FB000136843F480531360126802F48052019264
:100FC0000A6842F001020A60096801F0010101911A
:100FD000E02102910395049405960521069102A94A
:100FE000FFF7F6FD07B0F0BD1C4B9A42FAD1194A43
:100FF0001032136843F400431360126802F4004295
:1010000001920A6842F001020A600A6802F00102D5
:1010100001920A6842F004020A60096801F00401C2
:1010200001914FF40041029103950494059606271F
:10103000069702A9FFF7CCFD4FF4E050029003950C
:1010400004940596069702A90548FFF7C1FDC9E774
:10105000003001403038024000000240003C0040B7
:10106000000802402DE9F84F04468A4691461D4685
:10107000002694F85100012801D0022699E060680A
:101080004FF0040BB0F5827F01D1A06820B394F833
:10109000500001282BD04FF0010884F85080FFF752
:1010A0007FFE0746BAF1000F23D0B9F1000F20D020
:1010B00084F851B000206065C4F838A0A4F83C90D2
:1010C000A4F83E902063A086E08620646064A06857
:1010D000B0F5004F0FD018E084F851B04B4652469F
:1010E00051462046009500F033F9BDE8F88F022004
:1010F000FBE701265DE02068016821F04001016006
:101100002068016821F48041016020680168490677
:1011100003D4016841F040010160E068B0B133E000
:1011200020688168C90709D0007BA16B0870A06B9B
:10113000401CA063E08F401EE08707E0FFF730FE11
:10114000C01BA84201D3681C04D11DB1E08F002848
:10115000E6D11CE0032684F851802AE020688168EB
:10116000C90709D0C068A16B0880A06B801CA06370
:10117000E08F401EE08707E0FFF712FEC01BA84289
:1011800001D3681C0FD175B1E08F0028E6D13A4633
:101190002946204602F031F808B120206065606DD4
:1011A00028B1012605E0032684F8518001E084F887
:1011B0005180002084F85000304696E72DE9F84F22
:1011C00004468B4692461D46002694F8500001289E
:1011D0000DD04FF0010884F85080FFF7E1FD07467D
:1011E00094F85100B146012804D00226ACE0022058
:1011F000BDE8F88FBBF1000F1CD05FEA0A0019D0E0
:10120000032084F85100C4F85490C4F830B0A4F816
:1012100034A0A4F836A0C4F83890A4F83C90A4F800
:101220003E90C4F84490C4F84090A068B0F5004FD8
:1012300002D00BE0012687E02068016821F0400120
:1012400001602068016841F4804101602068016804
:10125000490603D4016841F040010160E068B0F53F
:10126000006F05D0606888B3BAF1010F2FD04FE04E
:10127000606810B1BAF1010F20D1206B216800889D
:10128000C860206B801C2063E08E401EE08615E065
:1012900020688168890709D5216B0988C160206BA6
:1012A000801C2063E08E401EE08607E0FFF778FD9B
:1012B000C01BA84201D3681C04D11DB1E08E0028D8
:1012C000E6D128E0032684F851803DE0FFE7206B5B
:1012D000216800780873206B401C2063E08E401E5C
:1012E000E08615E020688168890709D5216B0978B7
:1012F0000173206B401C2063E08E401EE08607E0F7
:10130000FFF74EFDC01BA84201D3681C0ED16DB182
:10131000E08E0028E6D13A462946204601F0B4FF87
:1013200008B120206065A06820B107E0032684F89A
:10133000518009E02068C16880680090606D08B144
:10134000012601E084F8518084F8509030464FE740
:101350002DE9FF4F81B004460E9E8B46984601252D
:10136000002794F8500001280ED0AA4684F850A017
:10137000FFF716FD814694F85100616801280DD0F1
:10138000B1F5827F08D103E0022005B0BDE8F08FFF
:10139000A16809B9042801D00227CFE0BBF1000FF2
:1013A0002DD0039858B35FEA080028D094F8510074
:1013B000042802D0052084F85100002060650399BC
:1013C000A163A4F83E80A4F83C80C4F830B0A4F82F
:1013D0003680A4F83480206460642068016849067F
:1013E00003D4016841F040010160E068B0F5006F8E
:1013F00007D06068F0B3B8F1010F49D07EE0012753
:101400009CE0606810B1B8F1010F3AD1206B2168FF
:101410000088C860206B801C2063E08E401EE08640
:101420002FE02068816889070DD5E18E59B1012D23
:1014300009D1216B0988C160206B801C2063E08E7C
:10144000401EE086002520688168C9070BD0E18F27
:1014500049B1C068A16B0880A06B801CA063E08FBD
:10146000401EE0870125FFF79BFCA0EB0900B0427E
:1014700007D300E00CE0701C03D0032784F851A0D0
:101480005CE0E08E0028CCD1E08F0028C9D13BE0A1
:10149000206B216800780873206B401C2063E08E6D
:1014A000401EE0862AE02068816889070DD5E18E1C
:1014B00059B1012D09D1216B09780173206B401CB2
:1014C0002063E08E401EE086002520688168C90701
:1014D0000BD0E18F49B1C068A16B0870A06B401CB4
:1014E000A063E08F401EE0870125FFF759FCA0EBC9
:1014F0000900B04201D3701C10D17EB1E08E0028EB
:10150000D1D1E08F0028CED14A463146204601F0A5
:10151000BBFE38B10127202060650FE0032784F867
:1015200051A00BE0A06818B92068C16880680090DD
:10153000606D08B1012701E084F851A0002084F813
:101540005000384621E710B5401EB0F1807F01D32E
:10155000012010BD4FF0E02460610F21601702F000
:10156000F9FD0020A06107202061002010BDFEE7EA
:1015700030B500224B68124CA468C4F30004114D2E
:10158000AD68C5F300052C430F4DAD68C5F30005EC
:101590002C4302D00122104630BD0C4D53B10C68D3
:1015A0001C43D1E902310B4341681C4329400C43E1
:1015B0004460F0E7436809682B400B434360EAE767
:1015C000002001400021014000220140E010FCFF0A
:1015D00030B500228368C3F30003002B02D0012240
:1015E000104630BD8C680B6823434468054D2C4081
:1015F000234343608368496823F400630B4383609B
:10160000EEE70000FFFEFFFC30B500224B68846867
:10161000C4F30004002C02D00122104630BD33B1C7
:1016200043688C6823F468432343436003E04368C2
:1016300023F468434360D1E9033423438468074DAE
:101640002C400D6805F070652C4323438360496886
:10165000C36A23F470030B43C362DEE7FDFCFFC0E3
:1016600010B54FF4407494FAA4F401F44073B4FA42
:1016700084F4E34000EB8300C36A01F01F011F24E0
:101680008C4002F01F02A3438A401343C36210BD83
:1016900070B54FF0007494FAA4F401F00073B4FA3A
:1016A00084F4E34000EB8300C4684FF0F87393FACE
:1016B000A3F501F0F871B5FA85F521FA05F50726CD
:1016C000AE4093FAA3F3B3FA83F3D940B4438A400C
:1016D0001443C46070BD000008B504490A680243A1
:1016E0000A6009680140009108BD000030380240DE
:1016F00008B504490A6802430A600968014000917C
:1017000008BD00003038024008B504490A680243A9
:101710000A6009680140009108BD000030380240AD
:1017200008B504490A6802430A600968014000914B
:1017300008BD00004038024008B504490A68024369
:101740000A6009680140009108BD0000403802406D
:1017500008B504490A6802430A600968014000911B
:1017600008BD000044380240034A1430515C0A5856
:1017700022F004020A5070478F790008034A515C36
:10178000425822F001024250704700008779000859
:10179000034A515C425842F0100242507047000028
:1017A0008F790008034A515C425842F001024250CE
:1017B000704700008F790008034B595C435823F0B1
:1017C00060631343435070478F790008044B001D3A
:1017D000595C0B586FF30F0313430B507047000015
:1017E0008F790008034B595C435823F0C00313431F
:1017F000435070478F790008034B595C435823F4DA
:1018000080631343435070478F790008034B595C42
:10181000435823F4C0431343435070478F79000863
:10182000034B595C435823F4907313434350704760
:101830008F790008034B595C435823F4007313431A
:10184000435070478F790008034B595C435823F489
:10185000C0531343435070478F790008034B595CC2
:10186000435823F440331343435070478F790008A3
:1018700030B500222B4C0379251F0168002B47D07F
:1018800099B343798BB1012B17D0022B1DD00122C4
:10189000817951B3234C0834231F01291DD002291B
:1018A00024D003292BD0012239E023688B43236005
:1018B00001682B680B432B60EAE72B688B432B6096
:1018C000016823680B432360E2E72B680B432B601E
:1018D000016823680B432360DAE7016825688D43BC
:1018E0002560006819680143196018E001681D68E7
:1018F0008D431D6000682168014321600FE001688D
:101900001D680D431D60006821680143216006E0E9
:101910002B688B432B60006821688143216010464F
:1019200030BD0000043C01402DE9F0410A6892FA04
:10193000A2F2B2FA82F30F2603258AE001249C402A
:101940002240002A7DD04C68012C01D0022C1BD1F2
:101950008C68876892FAA2FCBCFA8CFC4FEA4C0CAB
:1019600005FA0CFC27EA0C0792FAA2FCBCFA8CFCE4
:101970004FEA4C0C04FA0CF427438760CC684768A4
:1019800054439743274347600C69C76892FAA2FC07
:10199000BCFA8CFC4FEA4C0C05FA0CFC27EA0C074D
:1019A00092FAA2FCBCFA8CFC4FEA4C0C04FA0CF440
:1019B0002743C7604C68022C34D192FAA2F4B4FADF
:1019C00084F4082C16D24C69076A92FAA2FCBCFA7D
:1019D0008CFC4FEA8C0C06FA0CFC27EA0C0792FAF6
:1019E000A2FCBCFA8CFC4FEA8C0C04FA0CF42743E2
:1019F000076217E04F69D0F824C0140A94FAA4F8DB
:101A0000B8FA88F84FEA880806FA08F894FAA4F4B5
:101A1000B4FA84F4A4002CEA080CA7404CEA070CA2
:101A2000C0F824C04C68076892FAA2FCBCFA8CFC8F
:101A30004FEA4C0805FA08FC27EA0C0792FAA2F2D2
:101A400000E005E0B2FA82F25200944027430760BA
:101A50005B1C0A6832FA03F47FF470AF0020BDE823
:101A6000F0810069814301D0002070470120704758
:101A70000069814301D0002070470120704710B5F4
:101A8000044601F0B9F9206001F08CF9606001F0C2
:101A900097F9A060606801F0A1F9E06010BD10B591
:101AA00001220368C3F38013002B25D1D1E9002361
:101AB0001A43D1E9023423431A430B691A434B6991
:101AC0001A438B691A43CB691A430B6A1A4303689A
:101AD0004FF6BF74A3431A43026042684B6922F079
:101AE000040242EA134242600A6AB2F5005F02D180
:101AF000898C89B201610022C16921F40061C16150
:101B0000104610BD0149086070470000A400002085
:101B100010B501291CD004291CD010291CD0402943
:101B20001CD0B1F5807F1BD0B1F5806F1AD0062193
:101B30000D4B18305B5C184403680B4CE41D615C72
:101B400003248C40120CA3438A401343036010BD4E
:101B50000021EDE70121EBE70221E9E70321E7E7B7
:101B60000421E5E70521E3E77279000810B50129B2
:101B70001CD004291CD010291CD040291CD0B1F540
:101B8000807F1BD0B1F5806F1AD006210D4B183025
:101B90005B5C184403680B4CE41D615CF0248C40D2
:101BA000120CA3438A401343036010BD0021EDE7EC
:101BB0000121EBE70221E9E70321E7E70421E5E75B
:101BC0000521E3E77279000810B5012916D0042930
:101BD00016D0102916D0402916D0B1F5807F15D027
:101BE000B1F5806F14D00621036A0A4C615C0A24A7
:101BF0008C40A3438A401343036210BD0021F3E7E6
:101C00000121F1E70221EFE70321EDE70421EBE7F2
:101C10000521E9E78079000810B501291CD00429C5
:101C20001CD010291CD040291CD0B1F5807F1BD0BE
:101C3000B1F5806F1AD006210D4B18305B5C18444B
:101C400003680B4CE41D615C0C248C40120CA34314
:101C50008A401343036010BD0021EDE70121EBE74B
:101C60000221E9E70321E7E70421E5E70521E3E7AE
:101C7000727900082DE9F0410268264C264D274E66
:101C8000274F284B4FF0804CA04209D0604507D029
:101C9000A84205D0B04203D0B84201D0984205D145
:101CA000D1F8048022F0700242EA0802A0421BD060
:101CB000604519D0A84217D0B04215D0B84213D011
:101CC000984211D0184DA8420ED0184DA8420BD002
:101CD000174DA84208D0174DA84205D0164DA8426E
:101CE00002D0164DA84203D1CD6822F440722A4397
:101CF00002608A68C2620A888262A04201D0984269
:101D000001D109690163416941F00101416100208C
:101D1000BDE8F081000001400004004000080040E0
:101D2000000C00400004014000400140004401401C
:101D30000048014000180040001C00400020004006
:101D4000016921F490410161416921F02A01416159
:101D50007047143050E8001F41F0800140E8001245
:101D6000002AF7D170470C3050E8001F41F02001E5
:101D700040E80012002AF7D1704700002DE9FF412A
:101D800004460D4601270026E068C0F340300028D5
:101D900041D1E9686868AA69084329691143084381
:101DA000E16849F20C6291430843E060A868216948
:101DB00021F44051014321616869616921F4407156
:101DC000014361616846FFF75AFE1548844201D11C
:101DD000039E17E01348844201D1029E12E012488C
:101DE000844201D1029E0DE01048844201D1039E3D
:101DF00008E00F48844201D1029E03E00D4884426E
:101E000000D1029E3EB12B682BB1002731462046FF
:101E1000AA6900F011F804B03846BDE8F08100006E
:101E20000010014000440040004800400014014000
:101E3000004C0040005000402DE9F04104461927B5
:101E4000A1FB0778002064253226B2F5004F2BD085
:101E50009C469B0F4FEA8C0238464146FEF72CFA0F
:101E60000146B0FBF5F06FF01802504301EB800023
:101E700006EB0010B0FBF5F000F0F002B1FBF5F05E
:101E800002EB0012B1FBF5F06FF01803584301EBC1
:101E9000800006EB0010B0FBF5F000F00F001044DE
:101EA00080B2A060BDE8F081DA1840EB000338464C
:101EB0004146FEF701FA0146B0FBF5F00201B1FB25
:101EC000F5F06FF01803584301EB800006EBC000FB
:101ED000B0FBF5F000F0F80002EB4002B1FBF5F0CA
:101EE000584301EB800006EBC000B0FBF5F000F0BA
:101EF0000700104480B2A060D4E708B54FF0E0219D
:101F00000A690092421C05D0401C03E00A69D20312
:101F100000D5401E0028F9D108BD000010B58EB0D4
:101F200001228DF8042040F080008DF80500032088
:101F30008DF80610014601A800F05FFE8DF807003D
:101F4000010A05208DF80810084C228A052A00D3C2
:101F50000246628201A9E068FEF707FB628A044834
:101F6000E16804F085FB0EB010BD0000C80600203B
:101F70000048004010B512494FF48000886101F01C
:101F800021FA104C012020700A2003F013FF01F009
:101F90002BF9FEF7C1FD022020700A2003F00AFF92
:101FA00001F022F9FEF7B8FD032020700A2003F0AB
:101FB00001FF01F019F9BDE81040FEF7ADBD0000CA
:101FC000001002402401002030B593B0002410948A
:101FD0001194129414210BA8FEF70CFB079408949B
:101FE00009940A94182101A8FEF704FB4FF48075A8
:101FF0005148016841F480710160006800F480700C
:1020000000904D481438016841F0010101600068FA
:1020100000F0010000900720019003200290059439
:1020200001A94648FFF780FC4549464802788A588E
:10203000037822F06062CA5002788A58037822F04E
:10204000C002CA5002788A58037822F44032CA503B
:1020500002788A58037822F4907242F48072CA504F
:1020600002788A58037822F40072CA5002788A589B
:10207000037842F48062CA5002788A58037822F4C6
:10208000C05242F40062CA5002788A58037822F49F
:10209000C04242F40052CA502949027814315258C1
:1020A000007822F004024250109411941295264DAB
:1020B00010A92846FFF78CFA0B944FF400100C90EF
:1020C0000D940E944FF440700F900BA92846FFF723
:1020D0009BFAA86820F48060A8604FF480300790D5
:1020E000089407A91948FFF743FA4FF000742246F5
:1020F00021142846FFF7B4FA072221462846FFF7A5
:10210000C7FA134C40F2052122462846FFF7A8FAE9
:10211000072221462846FFF7BBFA0E4C40F20A215F
:1021200022462846FFF79CFA072221462846FFF759
:10213000AFFA13B030BD0000443802400000024046
:10214000006402406A790008002001400023014039
:10215000010030020200600210B54FF48000FFF76A
:10216000C7FA4FF40010FFF7C3FA01F0B3FF0122E2
:10217000002100F0CAFD01460E2001F0BBFF0E2039
:1021800001F080FF01F0A6FF0122022100F0BDFD59
:102190000146112001F0AEFF112001F073FF01F0A4
:1021A00099FF0122022100F0B0FD0146382001F024
:1021B000A1FF382001F066FF01F08CFF012202210F
:1021C00000F0A3FD0146392001F094FF392001F011
:1021D00059FF01F07FFF0122022100F096FD014628
:1021E000452001F087FFBDE81040452001F04ABFBF
:1021F0002DE9F04F89B0002407940894182101A814
:10220000FEF7F8F91020FFF767FA0420FFF764FAE9
:102210008020FFF761FA0120FFF75EFA0220FFF746
:102220005BFA0820FFF758FADFF8E8817848C8F829
:1022300018004FF47860C8F81800DFF8E09176488D
:10224000C9F81800DFF8D8A14FF08C70CAF8180050
:10225000DFF8D4B17348CBF81800754F7348B861F4
:102260003C2001900125029503940494059501A951
:102270004046FFF759FB4FF6C0700190029503945A
:102280000494059401A94046FFF74EFB4EF23E0030
:102290000190029503940494059401A94846FFF720
:1022A00043FB01950294059401A94846FFF73CFBC6
:1022B00018200190029503940494059401A95046B6
:1022C000FFF732FB40F60740019002950394049417
:1022D000059401A95846FFF727FBA80201900326A1
:1022E0000296059401A93846FFF71EFB4FF4625091
:1022F0000190029503940494059501A93846FFF7CF
:1023000013FB4CF21600019002950394049405947B
:1023100001A93846FFF708FB3002019002950394AB
:102320000494059501A94846FFF7FEFA280201909A
:10233000029503940494059501A95046FFF7F4FA19
:10234000F00201900296059401A95046FFF7ECFABD
:1023500001950294059501A93846FFF7E5FA382062
:102360000190029503940494059501A95846FFF73E
:10237000DBFA680201900296059401A95846FFF71E
:10238000D3FA01960296059401A94046FFF7CCFACC
:10239000284801684FF4704292FAA2F2B2FA82F22F
:1023A00021F4704106FA02F2114301604FF008086F
:1023B000CDF81C808DF820508DF821408DF82250EA
:1023C00007A8FFF755FAF86898FAA8F1B1FA81F171
:1023D000490006FA01F1884398FAA8F1B1FA81F1AF
:1023E000490004FA01F10843F860386898FAA8F146
:1023F000B1FA81F149008E4098FAA8F1B1FA81F161
:102400004900B0438C402043386009B0BDE8F08FEC
:1024100000007CF00010024000003EE30008024093
:102420000000024000003F0C00040240000096F84B
:10243000000C0240083801400C480B4901604FF481
:102440008271416000218160C160016141614FF48E
:10245000007282611822C2610162416281620A21B6
:10246000C162FEF733BD000000300140D8010020FA
:1024700010B592B0282108A8FEF7BCF8182102A8D0
:10248000FEF7B8F81E48016841F480410160006819
:1024900000F4804001901A481038016841F00201B0
:1024A0000160006800F0020001904FF4704002905B
:1024B0000220039003200490002405940694052034
:1024C000079002A90F48FFF72FFA08944FF4827083
:1024D00009900A940B940C944FF480200D900E9464
:1024E0000F9410940A201190074C08A92046FFF77A
:1024F000D6FA616821F01001616012B010BD0000D1
:1025000040380240000402400038004010B5114835
:102510000F4901604FF48271416000218160C16008
:10252000016101224261920482613822C26101622A
:10253000416281620A21C162FEF7C8FC0548FEF7CC
:10254000C5FC002803D0BDE81040FEF7A6BA10BDB8
:10255000003C00403002002010B586B0142101A8D4
:10256000FEF748F80220FFF7DBF818480068C0F3D0
:1025700002200122022100F0E1FB01461D2001F0B2
:10258000C9FD1D2001F08BFD5320ADF80400002093
:10259000029040F2E731039104900D4C01A92046CE
:1025A000FFF768FB206840F080002060A06844F2DC
:1025B00007018843A060606820F070006060A06838
:1025C00020F08000A06006B010BD00000CED00E01F
:1025D0000004004030B58DB0142108A8FEF70AF8B9
:1025E000182102A8FEF706F80420FFF799F83A48E8
:1025F000016841F002010160006800F002000190F2
:102600004FF4E0700290022003900024049405949B
:102610000694079002A93148FFF786F9ADF82040EB
:1026200009944FF6FF700A900B942D4C08A9204690
:10263000FFF720FB206820F080002060A06820F0D9
:10264000070040F00300A060A5132A4601212046A0
:10265000FFF75EFA002201212046FFF7DDFA002293
:1026600001212046FFF782FA002201212046FFF7D0
:10267000ABFA2A4610212046FFF74AFA0022102121
:102680002046FFF7C9FA002210212046FFF76EFA14
:10269000002210212046FFF797FA606820F07000B2
:1026A0006060A06820F08000A0602A46A515294639
:1026B0002046FFF72DFA002229462046FFF7ACFA04
:1026C000002229462046FFF751FA002229462046DB
:1026D000FFF77AFA0DB030BD3038024000040240F6
:1026E0000008004010B586B0142101A8FDF782FF54
:1026F0002020FFF715F815480068C0F302200022DB
:10270000114600F01BFB0146372001F003FD372086
:1027100001F0C5FC44F29F10ADF8040000200290C7
:10272000092003900A4C01A92046FFF7A3FA20686C
:1027300040F080002060606820F070006060A06859
:1027400020F08000A06006B010BD00000CED00E09D
:10275000001400402DE9F0418EB01C2107A8FDF7C0
:1027600049FF182101A8FDF745FF1020FEF7F0FFF3
:102770000120FEF7C9FF4FF4007001900225029579
:102780000327039700240494059407260696DFF890
:10279000708001A94046FFF7C7F8680201900295D2
:1027A0000397049401200590069601A94046FFF77F
:1027B000BBF801F097FC0122022100F0D8FA014693
:1027C000252001F0B7FC252001F076FC4FF4E13024
:1027D0000790089409940A940C200B900C940D9483
:1027E000084C07A92046FFF7C9FA2046FFF7A8FAC8
:1027F000E16841F40051E1600EB0BDE8F0810000F5
:1028000000000240001001402DE9F0418EB01C2173
:1028100007A8FDF7EFFE182101A8FDF7EBFE4FF426
:102820000030FEF789FF0820FEF76EFF20200190A0
:102830000225029503270397002404940594072694
:102840000696DFF8CC8001A94046FFF76DF84020DE
:10285000019002950397049401200590069601A922
:102860004046FFF761F8AA062A4D06212846FEF7E2
:10287000A3FF402206212846FEF7B4FF00220621CE
:102880002846FEF7EBFFAA1506212846FEF7C8FFEB
:10289000002206212846FEF7CDFF2A1506212846EC
:1028A000FEF7AAFF002206212846FEF7CDFF0022F0
:1028B00006212846FEF7AAFF06212846FEF754FF08
:1028C00001F010FC0122022100F051FA01462620FD
:1028D00001F030FC262001F0EFFB4FF4164007908A
:1028E000089409940A940C200B900C940D940A4CB3
:1028F00007A92046FFF742FA2046FFF721FAE168D0
:1029000041F40051E16004F0ADF80EB0BDE8F08193
:10291000000C024000600240004400402DE9F041FC
:102920008EB01C2107A8FDF765FE182101A8FDF750
:1029300061FE4FF48020FEF7FFFE0820FEF7E4FE64
:102940004FF480700190022502950326039600241F
:102950000494059407270697DFF8E08001A9404614
:10296000FEF7E2FF280201900295039604940120ED
:102970000590069701A94046FEF7D6FFAA06304DFE
:1029800003212846FEF718FF402203212846FEF7C0
:1029900029FF002203212846FEF760FF00220321C1
:1029A0002846FEF73DFF002203212846FEF742FF9E
:1029B0002A1503212846FEF71FFF0022032128467F
:1029C000FEF742FF002203212846FEF71FFF0321E6
:1029D0002846FEF7C9FE01F085FB0122002100F028
:1029E000C6F90146272001F0A5FB272001F064FB72
:1029F0004FF4E1300790089409940A940C200B904E
:102A00000C940D940F4C07A92046FFF7B7F9204608
:102A1000FFF796F9E06840F40050E060201D0A4995
:102A2000074AC978083288502046FFF792F90321F7
:102A30002846FEF7ADFE0EB0BDE8F081000C024066
:102A400000600240004800408F7900082DE9F04105
:102A50008EB01C2107A8FDF7CDFD182101A8FDF7B8
:102A6000C9FD2020FEF774FE0420FEF74DFE402035
:102A700001900225029503260396002404940594F0
:102A800008270697DFF8608101A94046FEF74CFF52
:102A900080200190029503960494012005900697EA
:102AA00001A94046FEF740FF504D4FF020663246E8
:102AB00001212846FEF780FE002201212846FEF76C
:102AC00091FE002201212846FEF7C8FEAF153A46C6
:102AD00001212846FEF7A4FE002201212846FEF728
:102AE000A9FE4FF48068424601212846FEF784FE85
:102AF000002201212846FEF7A7FE002201212846D8
:102B0000FEF784FE01212846FEF72EFE32460621FE
:102B10002846FEF751FE402206212846FEF762FEB7
:102B2000002206212846FEF799FE3A46062128464D
:102B3000FEF776FE002206212846FEF77BFE42467F
:102B400006212846FEF758FE002206212846FEF7F9
:102B50007BFE002206212846FEF758FE0621284665
:102B6000FEF702FE01F0BEFA0122022100F0FFF89A
:102B70000146472001F0DEFA472001F09DFA4FF4AC
:102B800016500790089409940A940C200B900C940A
:102B90000D94174E07A93046FFF7F0F83046FFF7BF
:102BA000CFF8F06840F40050F06006F10C0454E8EF
:102BB000000F40F0100044E800010029F7D10C4854
:102BC000001D0C49094A8979083288503046FFF7C0
:102BD000C0F806212846FEF7DBFD3046FFF7C3F8B4
:102BE0000EB0BDE8F0810000000802400064024021
:102BF000001401408F790008FEE730B503464FF618
:102C0000FF70002B15D0814213D04AF201040DE071
:102C100013F8012B50400022C50702D04008604045
:102C200000E04008521CD2B2082AF5D3491E89B2EE
:102C3000EED230BD30B4002848D0022946D3037804
:102C400042781446012B01D0002B3FD1891E052A62
:102C500037D008DC012A11D0022A14D0032A17D059
:102C6000042A06D119E0062A1CD00F2A1FD0102AE8
:102C700022D0204630BC0121FFF750B930BC89B2C8
:102C8000801C00F019B930BC89B2801C00F08AB9F0
:102C900030BC89B2801C00F0F7B930BC89B2801C0E
:102CA00000F04ABA30BC89B2801C01F051B930BC86
:102CB00089B2801C01F00AB830BC89B2801C01F0D6
:102CC00085B830BC89B2801C01F0FEB830BC7047BA
:102CD00070B50C4D2868E988022911D3421812F802
:102CE000023D527843EA0224891E89B2FFF785FF2C
:102CF000844205D1E9882868BDE87040FFF79ABF93
:102D000070BD0000C8060020FEE730B500F00703E4
:102D1000C3F10704042C00D90424181D072801D28C
:102D2000002300E0DB1E012505FA04F0401E0840E8
:102D300098409D406D1E1540284330BD30B500F0D1
:102D40000703C3F10704042C00D90424181D072825
:102D500001D2002300E0DB1E012505FA04F0401E2D
:102D6000084098409D406D1E1540284330BD30B549
:102D700000F00703C3F10704042C00D90424181D34
:102D8000072801D2002300E0DB1E012505FA04F02C
:102D9000401E084098409D406D1E1540284330BDA0
:102DA000704700000449096801F0F001034A09096D
:102DB000515CC8407047000008380240977900080D
:102DC0000449096801F4E051034A02EB91210978B2
:102DD000C840704708380240A779000804490968CC
:102DE00001F46041034A02EB51310978C840704751
:102DF00008380240A77900080748006800F00C0175
:102E00000648002907D0042904D0082903D1082046
:102E100000F008B802487047083802400024F40067
:102E200000127A0010B504460020104B196801F416
:102E300080020F49002A03D0B2F5800F00D149105B
:102E4000082C11D1186800F03F00B1FBF0F01968B0
:102E5000C1F388114843196801F44031012202EBA3
:102E600011414900B0FBF1F010BD000004380240F0
:102E70000024F40038B50C460D4A0023D3600C3210
:102E80001070FDF791FD0A2002F094FF084A01201E
:102E900010320090631C111F0648FEF759FA18B152
:102EA00000F090FA012038BD00F08CFA002038BD07
:102EB00024010020D80100202DE9F04F8FB00446F6
:102EC0004FF0000A342101A8FDF794FB60782178C7
:102ED00040EA0129E078A17840EA0127B9F11F0F03
:102EE00057D807EB0900202853D8F81DC0F3C70BAB
:102EF00001208DF804008DF8050003248DF806B03C
:102F000000264FF0000824E001A80021015500250B
:102F100009EB060080B20EA9FDF7D2FD01AA9DF8CB
:102F20003810105DA94008431055761CB6B2BE4259
:102F300002D34FF0010A03E06D1CEDB2082DE7D378
:102F4000641CE4B2BAF1010F05D008F1010808F0E1
:102F5000FF08D845D8D3214601A8FFF74EFE01ABA4
:102F6000611CC9B21855040A481CC2B25C540B4C0F
:102F7000208A904200D20246628201A9E068FDF7F1
:102F8000F4FA628A0648E16803F072FB0FB0BDE80C
:102F9000F08F02210120FEF7C1FFF7E7C8060020ED
:102FA000004800402DE9F04F8FB04FF0000A417803
:102FB000027841EA0229C178807841EA0027B9F114
:102FC0000F0F58D807EB0900102854D8F81DC0F38C
:102FD000C70B01208DF8040002208DF805000324A2
:102FE0008DF806B000264FF0000824E001A800216B
:102FF0000155002509EB060080B20EA9FDF778FD0A
:1030000001AA9DF83810105DA94008431055761CA0
:10301000B6B2BE4202D34FF0010A03E06D1CEDB21E
:10302000082DE7D3641CE4B2BAF1010F05D008F112
:10303000010808F0FF08D845D8D3214601A8FFF7BA
:10304000DCFD01AB611CC9B21855040A481CC2B2B0
:103050005C540B4C208A904200D20246628201A945
:10306000E068FDF782FA628A0648E16803F000FB37
:103070000FB0BDE8F08F02210220FEF74FFFF7E707
:10308000C806002000480040F0B58DB0002845D0AB
:103090004178027841EA0225C178807841EA00232C
:1030A000581E0F283ED80F2D3AD8E818102837D8C8
:1030B00001206E468DF8000003208DF801005800B5
:1030C00003248DF8020000220CE0A81880B2FDF75E
:1030D000E7FC070A611CC9B237554C1CE4B27054B6
:1030E000521C92B29A42F0D321466846FFF785FD02
:1030F000611CC9B23055030A481CC2B273540C4C4F
:10310000208A904200D2024662826946E068FDF75A
:103110002CFA628A0748E16803F0AAFA0DB0F0BD04
:10312000022100E003210320FEF7F8FEF6E700008D
:10313000C806002000480040F0B58DB0002845D0FA
:103140004178027841EA0225C178807841EA00237B
:10315000581E18283ED8182D3AD8E818192837D8FC
:1031600001206E468DF8000004208DF80100580003
:1031700003248DF8020000220CE0A81880B2FDF7AD
:1031800097FC070A611CC9B237554C1CE4B2705455
:10319000521C92B29A42F0D321466846FFF72DFDA9
:1031A000611CC9B23055030A481CC2B273540C4C9E
:1031B000208A904200D2024662826946E068FDF7AA
:1031C000D4F9628A0748E16803F052FA0DB0F0BD05
:1031D000022100E003210420FEF7A0FEF6E7000034
:1031E000C80600200048004010B51E2000F048FD31
:1031F000BDE810400320FEF780BEF8B504464FF44A
:10320000827560684FF48063A8420AD1A068B0F567
:10321000004F01D0984204D12068066826F040068D
:1032200006606068A8421ED1A06898420DD00B4687
:10323000009200228021204600F064F808B3606DFF
:1032400040F0200060650320F8BD0B46009200228C
:103250000121204600F056F898B1606D40F0200042
:1032600060650320F8BD0B46009200220121204634
:1032700000F048F828B1606D40F020006065032040
:10328000F8BD0020F8BD00007CB504460E4615468A
:103290003346012202212046009500F033F828B180
:1032A000606D40F02000606503207CBD1348144928
:1032B0000068B0FBF1F04FF47A7148430190606808
:1032C000B0F5827F0DD13346002280212046009543
:1032D00000F018F878B1606D40F0200060650320C0
:1032E0007CBD019838B10198401E0190206880682B
:1032F000C0430006F5D500207CBD0000A4000020DE
:1033000000366E012DE9F84304460F4691461E46ED
:10331000089DFDF745FD401B351AFDF741FD804630
:1033200026480068C0F3CB30684300903AE0701C38
:1033300038D0FDF735FDA0EB0800A84203D215B147
:10334000009858B32BE02068416821F0E00141600B
:103350006068B0F5827F0BD1A068B0F5004F02D055
:10336000B0F5806F04D12068016821F04001016050
:10337000A06AB0F5005F09D12068016821F400510E
:1033800001602068016841F400510160012050345F
:103390006070002020700320BDE8F88300250098AD
:1033A000401E00902068806837EA000004D00020AA
:1033B0004845BCD10020EFE70120F9E7A400002038
:1033C0007047000020210948816110218161082196
:1033D0008161C903816120210548816110218161DA
:1033E0000821816108050349886170470010024087
:1033F00000040240000C02402DE9F04F2DED0C8B33
:1034000085B0402000F03CFC0120FEF776FD032152
:103410000020FFF72FFDFE4CE07803F082FE41EC28
:10342000180B9FEDFCCBB0EE4C1AF0EE6C1A9FED32
:10343000FBBBB0EE4B0AF0EE6B0A00F09DFEB0EE67
:10344000409AF0EE609AA07803F06BFE53EC192BD3
:1034500003F0B6FE41EC190B9FEDF2DBB0EE4B0A28
:10346000F0EE6B0AB0EE4D1AF0EE6D1A00F084FE2D
:10347000B0EE40AAF0EE60AA607803F052FE53EC82
:103480001A2B03F09DFE53EC192B03F071FB53EC48
:10349000182B03F06DFB03F0AFFD0190502000F0FE
:1034A000EFFB0120FEF729FD03210020FFF7E2FCDE
:1034B000E07803F036FE41EC180BB0EE4C1AF0EE5B
:1034C0006C1AB0EE4B0AF0EE6B0A00F055FEB0EE4F
:1034D000409AF0EE609AA07803F023FE53EC192B8B
:1034E00003F06EFE41EC190BB0EE4D1AF0EE6D1AC2
:1034F000B0EE4B0AF0EE6B0A00F03EFEB0EE40AAD2
:10350000F0EE60AA607803F00CFE53EC1A2B03F087
:1035100057FE53EC192B03F02BFB53EC182B03F045
:1035200027FB03F069FD0546B0EE4C1AF0EE6C1A6D
:10353000B0EE4B0AF0EE6B0A00F01EFEDFF8D09200
:10354000BA4CA9F11009B0EE408A99F80000F0EEEB
:10355000608A04EB4000B0F8400003F0E2FD53EC59
:10356000182B03F02DFE41EC180B284603F0D9FD73
:1035700053EC182B04F030F803F00EFD82464FF0A8
:1035800080718A4501DD8A4603E0A948824500DA58
:1035900082469FEDA81BB0EE4B0AF0EE6B0A00F0DE
:1035A000EBFD99F80000B0EE408A04EB4000F0EE2D
:1035B000608AB0F850104FF0000BA1FB0A020BFB21
:1035C0000A224FEAEA7501FB052103F059FD53EC8D
:1035D000182B03F089FB9FED991B53EC112B03F083
:1035E000C7FA03F0D9FC80469FED96ABB0EE4B0ACC
:1035F000F0EE6B0AB0EE4A1AF0EE6A1A00F0BCFD6B
:1036000099F80000B0EE408A04EB4000F0EE608ACA
:10361000018EA1FB0A020BFB0A2201FB052103F02C
:103620002FFD53EC182B03F05FFB41EC190BB0EEB0
:103630004D1AF0EE6D1AB0EE4B0AF0EE6B0A00F088
:103640009BFD99F80000B0EE408A04EB4000F0EEDC
:10365000608A008A03F065FD53EC182B03F0B0FD7F
:1036600053EC192B03F084FA04F0A6F80F46064633
:10367000764A0B21901BB94102DA16460B2707E068
:103680007348301A57F1070002DA714E6FF00707DE
:10369000B0EE4B8AF0EE6B8AB0EE4C1AF0EE6C1A7C
:1036A000B0EE480AF0EE680A00F066FDDFF86091BF
:1036B000B0EE409AA9F11009F0EE609A99F8000076
:1036C00004EB4000018C0022A1FB0A0302FB0A323A
:1036D00001FB052103F0D4FC53EC192B03F004FB90
:1036E00041EC1B0B9FED5BDBB0EE480AF0EE680A85
:1036F000B0EE4D1AF0EE6D1A00F03EFD99F80000A4
:10370000B0EE409AF0EE609A34F8100003F009FD34
:1037100053EC192B03F054FD53EC1B2B03F028FA48
:1037200004F04AF80D4604464C4A0321101BA941F7
:1037300002DA1446032507E04948201A55F1010032
:1037400002DA474C6FF0010500BF4FF000099FED12
:1037500045CBB8F5FA6F59DA9FED441BB0EE480A35
:10376000F0EE680A00F008FDB0EE40BAF0EE60BA84
:10377000504603F06EFC41EC100BB0EE481AF0EE30
:10378000681A00F0F9FC9FED3B9B51EC100B53ECD9
:10379000192B03F015FD53EC1B2B03F0A5FA03F0D6
:1037A000FBFB83469FED351BB0EE480AF0EE680A3E
:1037B00000F0E2FCB0EE40BAF0EE60BAA8F5FA60B4
:1037C00003F047FC814641EC100BB0EE481AF0EED6
:1037D000681A049100F0D0FC53EC192B51EC100B3B
:1037E00003F0EEFC53EC1B2B03F07EFA03F0D4FB4A
:1037F0008246B0EE491AF0EE691AB0EE480AF0EED1
:10380000680A00F0B9FCB0EE409A3BE09AE0000094
:1038100034010020000000000000204000000000F3
:10382000000000400000000000003040DC060020E6
:10383000000100FF00000000000037400000000011
:1038400000409F400000000000001C400000F4FF0A
:10385000F8FF0F000000000000002E400000FCFFF9
:10386000FEFF030000000000000010400000000008
:103870000080404000000000000008400000000000
:103880000000F03F0499F0EE609A41EC109BB0EE1E
:10389000481AF0EE681A00F06FFC9FED751B51ECB2
:1038A000100B53EC112B03F08BFC53EC192B03F092
:1038B0001BFA03F071FB814640F2DC5018EB000F5D
:1038C0003FDA08F2DC5003F0C4FBB0EE48BAF0EE89
:1038D00068BACDE9021041EC100BB0EE4B1AF0EED5
:1038E0006B1A00F049FC53EC1A2B51EC100B03F04F
:1038F00067FC41EC190B504603F0ABFB53EC192B62
:1039000003F036F903F048FB8246DDE9021041EC92
:10391000100BB0EE4B1AF0EE6B1A00F02DFC53ECCE
:103920001C2B51EC100B03F04BFC41EC190B4846DF
:1039300003F08FFB53EC192B03F01AF903F02CFB67
:10394000814646E09FED4C1BB0EE480AF0EE680A57
:1039500000F012FCB0EE409AF0EE609A504603F090
:1039600078FB41EC100BB0EE481AF0EE681A00F04C
:1039700003FC53EC1A2B51EC100B03F021FC53EC1D
:10398000192B03F0B1F903F007FB8346B0EE4C1A94
:10399000F0EE6C1AB0EE480AF0EE680A00F0ECFBAC
:1039A000B0EE409AF0EE609AA8F5FA6003F051FB91
:1039B00041EC100BB0EE481AF0EE681A00F0DCFB98
:1039C00053EC192B51EC100B03F08EF903F0E4FAD1
:1039D0008246A8EB0B00DFF8A880C8F80400B6EB1D
:1039E0000A0667EBEA77B4EB090465EBE975B0EE1C
:1039F0004D1AF0EE6D1AB0EE480AF0EE680A00F0CB
:103A0000BBFBB0EE409AF0EE609A3046394603F0C8
:103A100037FB41EC1A0B9FED1B1BB0EE480AF0EE92
:103A2000680A00F0A9FB01990022A4FB010305FB31
:103A3000013104FB0211B0EE408AF0EE608A03F01F
:103A40001FFB53EC182B03F04FF953EC1A2B03F028
:103A5000C3FD53EC192B03F047F903F09DFAC8F8A6
:103A6000080000BF05B0BDEC0C8BBDE8F08F000076
:103A700000000000000014400000000000804240F0
:103A8000240100200000000000003540FDF78EB941
:103A900070B52E48016821F0070141F00501016071
:103AA000016801F007010529FAD12949086840F4A5
:103AB000804008602748026842F480320260026851
:103AC000C2F34042002AFAD0224A234B121D146846
:103AD000224D2C4023431360136823F440331360BA
:103AE000026842F0807202600268C2F34062002AFB
:103AF000FAD04868C0F380300028FAD01548083062
:103B0000016821F0F0010160016821F4E05141F405
:103B1000A0510160016821F4604141F4004101605D
:103B2000016821F0030141F002010160016801F028
:103B30000C010829FAD10A48FDF7E4FF0020FDF73F
:103B400057F9002801D0FCF7A8FF70BD003C0240E7
:103B50000070004000380240042A40000080BFFF8F
:103B6000007A030A0248016841F47001016070475D
:103B700088ED00E02DE9F041374F3869C0F30000CF
:103B8000002863D0354E7068401C70600024012509
:103B9000042801DD35607460B068401CB0600928FD
:103BA0001FDDDFF8BC8098F80000062818D1D8F88F
:103BB0001800804798ED010A2A49B5EEC00AF1EED7
:103BC00010FA05DBBCEEC00A10EE100A088107E00F
:103BD000B1EE400ABDEEC00A10EE100A4042088164
:103BE000B4603069401C3061182801DDF560346133
:103BF000B069401CB061312801DD7561B461F069C4
:103C0000401CF061632806DDF4611748006806284F
:103C10001ED002F0CFFA706A401C7062B0F5967F39
:103C200001DB35627462F06A401CF062B0F5FA7F25
:103C300001DBB562F462706B401C7063B0F57A7F93
:103C400001DB356374636FF001003861BDE8F0811A
:103C500002F0EEFADFE70000000400405800002008
:103C6000A0070020AC0000202000002002F016BDBC
:103C7000704702F0D1B902F0B7BC02F05DBCFEE7BC
:103C800010B50D490022CA600C310870FCF78CFE9B
:103C90000A2002F08FF8084901231A460C31074820
:103CA000FDF78CFA18B1FFF78DFB012010BDFFF76F
:103CB00089FB002010BD000024010020D801002055
:103CC000014A22F810107047DE0000202DE9F04F65
:103CD0008FB0074600200E9082467878397840EA07
:103CE0000129F878B97840EA012838790D90A8F1CF
:103CF00001000F2861D80D98B8EBC00F5DD8B9F15D
:103D00001F0F58D809EB0800202854D8002500269A
:103D100021E0B81990F805B000240120A04010EA75
:103D20000B0F02D04FF47F4100E0002109EB0500AA
:103D300080B200F0ADF86D1CADB2454502D34FF036
:103D4000010A03E0641CE4B2082CE6D3BAF1010FC7
:103D500004D0761CF6B20D988642DAD30E99012271
:103D6000481CC0B26C460DF801200F22411CC9B29C
:103D7000225460183A680260091DCDB2294668468F
:103D8000FEF73BFF691CC9B26055030A481CC2B26A
:103D900063540C4C208A904200D2024662826946EB
:103DA000E068FCF7E2FB628A0748E16802F060FC29
:103DB0000FB0BDE8F08F022100E003210F20FEF7D5
:103DC000ADF8F5E7C806002000480040F0B58DB01A
:103DD00004460027002C4CD06078217840EA012668
:103DE000E078A17840EA01252079691E0F2944D89E
:103DF000B0EB450F41D10F2E3DD8701910283AD89D
:103E000000230BE004EB43008179407941EA002173
:103E1000F01880B2FFF754FF5B1C9BB2AB42F1D3AA
:103E20000121781CC0B26D460DF807101022411C0C
:103E3000C9B22A54681822680260091DCCB2214612
:103E40006846FEF7DAFE611CC9B22855030A481C11
:103E5000C2B26B540C4C208A904200D2024662825D
:103E60006946E068FCF781FB628A0848E16802F075
:103E7000FFFB0DB0F0BD022000E00320C1B2102016
:103E8000FEF74CF8F5E70000C806002000480040A7
:103E900010B51038C21700EB527323F00702801AD6
:103EA00001228240074CD810B1F57F4F05D0002980
:103EB00002D1215C9143215410BD215C1143215456
:103EC00010BD0000A800002010B58EB00446607838
:103ED000217840EA0120E178A27841EA0221002914
:103EE00008D0B1F57F4F05D003210520FEF716F865
:103EF0000EB010BD1F2824D8FFF7CAFF01208DF88F
:103F0000040005208DF805002068CDF80600062184
:103F100001A8FEF772FE8DF80A00010A08208DF84C
:103F20000B10094C228A082A00D30246628201A99A
:103F3000E068FCF71AFB628A0448E16802F098FB2B
:103F4000D6E70221D1E70000C80600200048004063
:103F500010B58EB00346002B2CD05878197840EA63
:103F60000120D9789A7841EA02210F2824D8FFF756
:103F7000A7FE01208DF8040006218DF805101868B1
:103F8000CDF8060001A8FEF738FE8DF80A00010AF8
:103F900008208DF80B100B4C228A082A00D3024609
:103FA000628201A9E068FCF7E0FA628A0648E168EB
:103FB00002F05EFB0EB010BD02210620FDF7AEFF41
:103FC000F8E70000C80600200048004004484FF40D
:103FD0000031816104218161082181617047000005
:103FE000000802402DE9F0410024194E4FF48020D2
:103FF000B0610A2001F0DEFE0420B0610A2001F069
:10400000D9FE01213046FDF733FD012800D10124FE
:1040100000254FF400276400B7610A2001F0CAFEB2
:104020000821B161052001F0C5FE01213046FDF7F0
:104030001FFD012801D144F00104052001F0BAFE62
:104040006D1CEDB20F2DE6D3A0B2BDE8F0810000EB
:104050000008024003B401984100009850EAC120D2
:1040600018BF04204A0D18BF40F0010040F2FF7253
:10407000B2EB515F08BF40F00200012808BF0520E5
:1040800002B07047002809DB00F01F0201219140B7
:104090004009800000F1E020C0F8001170470028BE
:1040A00009DB00F01F02012191404009800000F16E
:1040B000E020C0F800117047002809DB00F01F0263
:1040C000012191404009800000F1E020C0F800117A
:1040D0007047000002480068C0F3022070470000EB
:1040E0000CED00E002480068C0F3022070470000B9
:1040F0000CED00E00907090E002804DB00F1E020C8
:1041000080F80014704700F00F0000F1E02080F804
:10411000141D70470907090E002804DB00F1E02098
:1041200080F80014704700F00F0000F1E02080F8E4
:10413000141D70470907090E002804DB00F1E02078
:1041400080F80014704700F00F0000F1E02080F8C4
:10415000141D70470907090E002804DB00F1E02058
:1041600080F80014704700F00F0000F1E02080F8A4
:10417000141D7047000000002DE9F04D2DED040BDB
:104180002DED0C8B96B0DDE92350259CDDF888A041
:1041900025F0004624F00048BAF1000F14BF0121B9
:1041A000002101EB4502FE4953184A1093422AD3DD
:1041B000002814BF0123002303EB44030B44F949F7
:1041C0008B4220D358EA00019FEDF78B6FD0DFF8C8
:1041D000E0B35D4503D1BAF1000F05D187E0BAF134
:1041E000000F08BF002100D0012101EB450111F5AE
:1041F000001F08D8002814BF0121002101EB440151
:1042000011F5001F0BD99DED241B9DED220B16B05F
:10421000BDEC0C8B04B0BDE8F04D00F05DBE002796
:10422000002DBCBFE349884521DAE3498845A8BF92
:1042300002271CDAC3451ADCE04901EB2851142996
:1042400008DDC1F1340220FA02F101FA02F28242E1
:104250000DD108E058B9C1F1140228FA02F101FAAF
:1042600002F2424503D101F00101C1F1020756EA11
:104270000A011DD1002C1BDA002D18BF022F01D01E
:10428000012F0AD00220FCF7E4F916B0BDEC0C8B2C
:1042900004B0BDE8F04D00F007BE0220FCF7D9F9EC
:1042A00000F002FE51EC100B02F056FC83E01EE021
:1042B0009FEDC39B9FEDC4AB002872D1BD488045E4
:1042C0002DD105F1804010F5801008BFBAF1000F24
:1042D0000DD0B34515DC002CA1BF9DED240B16B00D
:1042E000BDEC0C8B04B0A8BFBDE8F08D12E0B0EEC1
:1042F000480AF0EE680A16B0BDEC0C8B04B0BDE8BD
:10430000F08D002C06DA9DED240B51EC100B02F021
:1043100023FC50E0AE48784490ED000BEBE7D84525
:104320004FD1002C4ADA2EB186423BD1BAF1000FB0
:1043300044D126E0BAF1000F13D00220FCF789F92E
:1043400000F0E6FD8DED020B9DED220B8DED000BD7
:1043500010EE900A039961F31E0003909DED020B8D
:10436000C9E78DED029B9DED220B19EE901A10EE20
:10437000900A8DED000B61F31E0003909DED020B82
:10438000B9E78DED02AB9DED220B1AEE901A10EEFF
:10439000900A8DED000B61F31E0003909DED020B62
:1043A000A9E729E00ADA9DED220B51EC180B53EC3A
:1043B000102B02F099FC41EC100B9CE79DED220BB9
:1043C00099E7864218DAB4F1804F0DD0A4F100507D
:1043D000B0F1FF5010D1002D0EDB9DED220B51EC02
:1043E000100B02F033FAE6E79DED220B53EC102B95
:1043F00051EC100B00F0AEBC9DED220B51EC100BFC
:1044000001F0DEFCBAF1000FCDE90C0134D19FEDD3
:10441000720BDEB1A6F1E040B0F17F602CD1002D2F
:1044200001DD002C0DDA002D01DD002C1FDB002D3D
:1044300016DA002C14DB012F08BF9FED690B3FF447
:104440005AAFB0EE490AF0EE690A54E7022F18BFDE
:10445000002D0CD0012F0AD1002DFFF64CAF06E045
:10446000002DB8BF002C07DA012F3FF444AFB0EEA7
:104470004A0AF0EE6A0A3EE7012000EBE57A5AEAC2
:1044800007000CD05848002580457CDD5749584826
:10449000884514DDB0420DDB002C19DB2BE0012038
:1044A000FCF7D7F816B0BDEC0C8B04B0BDE8F04DAE
:1044B00000F01EBDB34502DC002C09DC1BE0864287
:1044C00002DA002C17DA03E05E4527DD002C12DD4E
:1044D0000220FCF7BEF800F01BFD10EE901A19EE5A
:1044E000900A8DED020B8DED009B61F31E00039091
:1044F0009DED020BFFE60220FCF7ABF800F018FD83
:1045000010EE901A18EE900A8DED020B8DED008BD7
:1045100061F31E0003909DED020BECE69DED220B76
:1045200053EC182B51EC100B03F056F89FED320BA7
:10453000CDE90A0153EC102B9DED0A0B51EC100B49
:1045400002F03EFE9FED2E1B53EC112B02F06CFF90
:104550009DED0A1B53EC112B02F032FE9FED2A1B3E
:1045600053EC112B02F060FF9DED0A0B41EC190B8F
:1045700053EC102B51EC100B02F022FE53EC192BD4
:1045800002F01EFE00E07EE09FED210B41EC1A0BD5
:1045900053EC102B9DED0A0B51EC100B3CE000008E
:1045A000FFFF1F00FFFF0F00000000000000F03FB2
:1045B0000000F03F0000F07F0000404301FCFFFFDF
:1045C000000000000000F07F00000000000000007C
:1045D0005E370000000000000000000000000080C6
:1045E000000000000000F0FF0000E0410000F04388
:1045F000FFFFEF3F00000000000000000000D03F80
:10460000555555555555D53F000000000000E03F79
:10461000000000604715F73F02F0D2FD41EC190B96
:104620009FEDFD0B51EC1A0B53EC102B02F0C8FD63
:1046300041EC1A0B9FEDFA0B53EC102B9DED0A0B7E
:1046400051EC100B02F0BCFD53EC1A2B02F0C4FF2E
:1046500041EC1A0B51EC190B53EC1A2B02F088FAAF
:104660000690CDE906519DED060B53EC192B51EC4C
:10467000100B02F0B1FF53EC1A2B02F0D5FE41EC07
:10468000100B00F09FB90020B6F5801F0EDA9FEDE9
:10469000E60B53EC102B9DED0C0B51EC100B02F0C4
:1046A0008FFDCDE90C016FF034000E4600EB265073
:1046B000A0F2FF38C6F31300DD4940F07F6646F0F4
:1046C00040568842D8BF002409DDDA498142C8BF7C
:1046D000012404DC0024A6F5801608F10108D64860
:1046E000784400EBC4000D9690ED00BB9DED0C0BE3
:1046F00053EC1B2B51EC100B02F06EFF9DED0C0BDD
:1047000041EC1A0B53EC1B2B51EC100B02F030FA5E
:1047100041EC100B51EC180B53EC102B02F0E4FAA7
:1047200041EC1C0B51EC1A0B53EC1C2B02F048FD16
:1047300041EC190BC1488DED109B7844109590ED1C
:10474000000B4FF0005040EA660000EB84408DED16
:104750000A0B00F500200B909DED0A0B53EC1B2B70
:1047600051EC100B02F038FF9DED0C1B53EC112B9C
:1047700002F05AFE41EC100B53EC102B9DED100B88
:1047800051EC100B02F01CFD9DED0A0B41EC1B0BD4
:1047900053EC102B9DED100B51EC100B02F010FDA3
:1047A00053EC1A2B02F040FE53EC1B2B02F014FFCB
:1047B00053EC1C2B02F004FD41EC1B0B53EC192BAA
:1047C00051EC190B02F0FCFC41EC1A0B9C48062141
:1047D000B0EE4A0AF0EE6A0A784400F0E9FAB0EE68
:1047E00040CAF0EE60CA53EC1A2B51EC1A0B02F0DF
:1047F000E7FC53EC1C2B02F0E3FC9DED100B41ECAD
:104800001A0B53EC192B51EC100B02F0B1F953ECCD
:104810001B2B02F0D5FC53EC1A2B02F0A9F99DEDED
:10482000100B41EC1A0B53EC102B51EC100B02F057
:10483000C7FC41EC1C0B9FED84DB53EC1D2B02F0FD
:1048400097F953EC1A2B02F093F90A90CDE90A512B
:104850009DED0A0B53EC1D2B51EC100B02F0BCFE2E
:1048600053EC1C2B02F0B8FE53EC1A2B02F0DCFDCB
:104870009DED0A0B41EC1C0B53EC102B9DED100B26
:1048800051EC100B02F09CFC41EC1A0B53EC192B71
:1048900051EC1C0B02F094FC9DED0A0B41EC190B42
:1048A00053EC102B51EC1B0B02F08AFC53EC192B30
:1048B00002F05EF941EC190B51EC1A0B53EC192B79
:1048C00002F056F91090CDE910519DED100B53EC0C
:1048D0001A2B51EC100B02F07FFE53EC192B02F057
:1048E000A3FD41EC190B9FED5A0B53EC102B9DEDE2
:1048F000100B51EC100B02F063FC41EC1A0B9FED16
:10490000560B51EC190B53EC102B02F059FC41ECF7
:10491000190B9FED530B53EC102B9DED100B51EC2D
:10492000100B02F04DFC53EC192B02F021F941EC75
:10493000100B4D48784400EBC40090ED001B51EC87
:10494000100B53EC112B02F013F941EC190B4046FC
:1049500002F07FFBCDE90A0153EC192B51EC1A0B45
:1049600002F006F941EC100B4048784400EBC4001B
:1049700090ED00BB51EC100B53EC1B2B02F0F8F840
:104980009DED0A1B53EC112B02F0F2F80690CDE9D5
:1049900006519DED0A0B53EC102B9DED060B51ECCF
:1049A000100B02F019FE53EC1B2B02F015FE53EC1A
:1049B0001A2B02F011FE53EC192B02F035FD41ECDD
:1049C000100B00BF781EB0EE48AAF0EE68AA5AEAB3
:1049D000000008BF9FED268B9DED241B53EC102B90
:1049E0008DED001B00959DED240B51EC100B02F09A
:1049F000E7FB9DED000B41EC190B53EC102B9DEDEB
:104A0000240B51EC100B02F0E7FD9DED061B53EC5F
:104A1000112B02F0D5FB2FE0FE822B654715F73FE7
:104A200044DF5DF80BAE543E000000000000404340
:104A30008E9803007AB60B000C3300003A33000066
:104A400044320000000000000000000000000840A8
:104A5000000000E009C7EE3FFD033ADC09C7EE3F66
:104A6000F5015B14E02F3EBED8300000923000000C
:104A7000000000000000F0BF53EC192B02F078F8A2
:104A80009DED060B41EC190B53EC102B9DED000B2B
:104A900051EC100B02F094FBCDE910019DED100BD1
:104AA00051EC190B53EC102B02F062F8CDE9020126
:104AB0000C46AB498C422FDB611A084318D19DED9F
:104AC000100B53EC102B9DED020B51EC100B02F070
:104AD00083FD41EC1B0B9FEDA40B51EC190B53EC28
:104AE000102B02F045F853EC1B2B02F067FC2DD283
:104AF0000220FBF7AEFD00F00BFA10EE901A18EE54
:104B0000900A8DED020B8DED008B61F31E0003907A
:104B10009DED020BFFF7EFBB954A24F00041914257
:104B200014D39449214408437FF4E5AC9DED100B68
:104B300053EC102B9DED020B51EC100B02F04CFDD1
:104B400053EC192B02F03AFC7FF6D5AC24F0004070
:104B500089498A4A002601EB205182422BDA481CFF
:104B60004FF4801121FA00F02044854AC0F30A5125
:104B70007A44A1F2FF3192ED000B824A8DED0A0BCF
:104B8000CA4020EA0202C0F3130040F48010C1F1D1
:104B9000140120FA01F60B92002CB8BF76429DED6D
:104BA0000A0B53EC102B9DED100B51EC100B02F087
:104BB00013FDCDE910019DED100B51EC190B53ECD9
:104BC000102B01F0D5FF9FED700B0A90CDE90A5133
:104BD00053EC102B9DED0A0B51EC100B02F0F0FA88
:104BE00041EC1B0B9FED6A0B53EC102B9DED0A0B58
:104BF00051EC100B02F0E4FA9DED100B41EC1C0B94
:104C000053EC102B9DED0A0B51EC100B02F0E4FC61
:104C100053EC192B02F008FC9FED5F1B53EC112B9A
:104C200002F0CEFA53EC1C2B01F0A2FF41EC190B61
:104C300051EC1B0B53EC192B01F09AFFCDE902014B
:104C40009DED020B53EC1B2B51EC100B02F0C4FC3E
:104C500053EC192B02F0E8FB9DED020B41EC190B14
:104C600053EC102B51EC100B02F0AAFACDE90A011B
:104C70004B489DED0A0B0521784400F099F89DED15
:104C80000A1B51EC100B53EC112B02F099FA9DED1D
:104C9000021B53EC112B02F0C7FBCDE906019DED81
:104CA000020B53EC192B51EC100B02F089FA53EC68
:104CB000192B01F05DFF9FED3C0B41EC190B53EC00
:104CC000102B9DED060B51EC100B02F085FC9DEDB9
:104CD000060B41EC1B0B53EC102B9DED020B51EC22
:104CE000100B02F06DFA53EC1B2B01F0FDFF53EC9F
:104CF000192B02F071FC9DED021B53EC112B02F0FD
:104D00006BFC53EC1A2B02F08FFBCDE9020101EB97
:104D1000065001150029C8BF039015DC9DED020B5C
:104D2000324651EC100B02F0DAFDFFF793F904283C
:104D300008BF00F0FDF832469DED020B51EC100B60
:104D400002F0CDFDCDE902019DED020B51EC180BF7
:104D500053EC102B02F034FAFFF72DBB00000000DB
:104D60000000904000000000FE822B654715973C34
:104D700000CC904000346F3F01FCFFFF0000E03F9B
:104D8000042F0000FFFF0F0000000000432EE63F4D
:104D9000396CA80C615C20BEEF39FAFE422EE63F6A
:104DA000D42D0000000000000000000000000040C2
:104DB00070B504462DED028B4D1E00EBC500B0EE24
:104DC000408AF0EE608A90ED000B35F0060017D0B7
:104DD00053EC182B51EC100B02F0F2F941EC100BD4
:104DE0006D1E04EBC50090ED001B51EC100B53EC55
:104DF000112B01F0BDFE41EC100B35F00600E7D1A0
:104E0000022D36D0042D1CD0062D1CBFBDEC028B0C
:104E100070BD53EC182B51EC100B02F0D1F994ED4E
:104E20000A1B53EC112B01F0A3FE53EC182B02F0DC
:104E3000C7F994ED081B53EC112B01F099FE41ECDE
:104E4000100B53EC182B51EC100B02F0B9F994ED48
:104E5000061B53EC112B01F08BFE53EC182B02F0C8
:104E6000AFF994ED040B53EC102B01F081FE41ECF3
:104E7000100B53EC182B51EC100B02F0A1F994ED30
:104E8000021B53EC112B01F073FE53EC182B02F0B4
:104E900097F994ED001B53EC112B01F069FEBDEC6A
:104EA000028B41EC100B70BD9FED070B10B553EC5E
:104EB000102B9FED070B51EC100B01F015FF41EC8F
:104EC000100B10BD000000000000000000000000FA
:104ED000000000000000F03F10B553EC112B51EC26
:104EE000100B01F045FE41EC100B10BD000000005E
:104EF0009FED050B10B553EC102B51EC100B01F08E
:104F0000F3FE41EC100B10BD00000000000000009B
:104F10009FED050B10B553EC102B51EC100B02F06C
:104F20004FF941EC100B10BD0000000000000070B4
:104F30009FED050B10B553EC102B51EC100B02F04C
:104F40003FF941EC100B10BD000000000000001004
:104F50000149062008707047A007002030B5184AA4
:104F60001848111D03785B5804786FF30F0343F062
:104F7000030363501449144B4C33114D0478083526
:104F80006351124B04782D1D63510378D358047874
:104F900043F001031351202393600378D358007822
:104FA00043F010031350886840F00100886088685F
:104FB00040F080408860886840F44070886030BD70
:104FC000006402406A79000800200140500000207F
:104FD0002DE9F05F2DED068BFB498A6842F0804297
:104FE0008A609FEDFA8B44F288799FEDFA9ADFEDA3
:104FF000FA9A42F6E06544F62066DFEDF8AA9FEDE6
:10500000F8AAF84C40F6CA4840F6CC4A40F6C84BDD
:1050100040F6CB47082822D2DFE800F00484F6F5FA
:10502000F4F3F2F10120FBF7C5FB53EC182B51EC24
:10503000100B02F0C5F801F0DFFF80B2A0804845F8
:1050400011D8A0F56850BC3800EE100AB8EEC00ABE
:10505000C0EE090ABCEEE00A10EE100AA080BDEC1A
:10506000068BBDE8F09FA0F58E418939B9420ED874
:10507000481C00EE100AB8EEC00AC0EE090ABCEEE9
:10508000E00A10EE100A00F57A60A080E7E7A0F5CC
:10509000A8415539B9420ED8481C00EE100AB8EEA6
:1050A000C00AC0EE090ABCEEE00A10EE100A00F5D4
:1050B000FA50A080D3E7A0F5C241213941450DD86F
:1050C000481C00EE100AB8EEC00AC0EE290ABCEE79
:1050D000E00A10EE100A2844A080C0E7A0F5DA41EB
:1050E000EC3941450ED8481C00EE100AB8EEC00A53
:1050F000C0EE290ABCEEE00A10EE100A00F57A5064
:10510000A080ACE7A0F5F440B63800EE100AB8EE87
:10511000C00AC0EE290ABCEEE00A10EE100A3044C4
:10512000A0809CE70220FBF745FB53EC182B51ECC9
:10513000100B02F045F801F05FFF80B2E0804845B7
:105140000ED8A0F56850BD3800EE100AB8EEC00ABF
:10515000C0EE290ABCEEE00A10EE100AE0807EE7FD
:10516000A0F58E41893941450ED8481C00EE100A41
:10517000B8EEC00AC0EE290ABCEEE00A10EE100A32
:1051800000F57A60E0806AE7A0F5A841543941450E
:105190000ED8481C00EE100AB8EEC00AC0EE290A6C
:1051A000BCEEE00A10EE100A00F5FA50E08056E777
:1051B000A0F5C2411F3941450DD8481C00EE100A28
:1051C000B8EEC00AC0EE290ABCEEE00A10EE100AE2
:1051D0002844E08043E7A0F5DA41EA39594514D87C
:1051E000481C00EE100AB8EEC00AC0EE2A0ABCEE57
:1051F000E00A10EE100A00F57A50E0802FE7A9E2ED
:105200002BE2A9E12BE197E00FE0A0F5F440B238E2
:1052100000EE100AB8EEC00AC0EE2A0ABCEEE00AA0
:1052200010EE100A3044E08019E70320FBF7C2FAC1
:1052300053EC182B51EC100B01F0C2FF01F0DCFE17
:1052400080B2E08244F287719FED670A88420ED8EF
:10525000A0F56850B83800EE900AF8EEE00A80EE4B
:10526000801ABCEEC10A10EE100AE082F7E6A0F543
:105270008E41883940F6CE4291420ED8481C00EE4D
:10528000900AF8EEE00A80EE801ABCEEC10A10EE39
:10529000100A00F57A60E082E1E6A0F5A8415739EE
:1052A00040F6CD42914210D8481C00EE100AB8EEEC
:1052B000C00ADFED4E0A80EE201ABCEEC10A10EEE5
:1052C000100A00F5FA50E082C9E6A0F5C24125397E
:1052D00041450DD8481C00EE900AF8EEE00A80EE39
:1052E000801ABCEEC10A10EE100A2844E082B6E62D
:1052F000A0F5DA41F039B9420ED8481C00EE100A88
:10530000B8EEC00AC0EE0A0ABCEEE00A10EE100ABF
:1053100000F57A50E082A2E6A0F5F440BB3800EE3A
:10532000100AB8EEC00AC0EE0A0ABCEEE00A10EE9F
:10533000100A3044E08292E60420FBF73BFA53EC7B
:10534000182B51EC100B01F03BFF01F055FE80B221
:10535000208344F2897188420ED8A0F56850BC3889
:1053600000EE100AB8EEC00AC0EE0A0ABCEEE00A6F
:1053700010EE100A208372E6A0F58E418A3951455D
:105380000ED8481C00EE100AB8EEC00AC0EE0A0A99
:10539000BCEEE00A10EE100A00F57A6020835EE6AB
:1053A000A0F5A8415739514522D8481C00EE100AF3
:1053B000B8EEC00AC0EE0A0ABCEEE00A10EE100A0F
:1053C00000F5FA5020834AE600200140000000006A
:1053D00000002440FCA9513F9A99513FD578513F94
:1053E0005EBA513FAC00002023DB513FC1CA513FA0
:1053F000A0F5C2412439B9420DD8481C00EE100A6C
:10540000B8EEC00AC0EE090ABCEEE00A10EE100ABF
:105410002844208323E6A0F5DA41F039B9420ED8BA
:10542000481C00EE100AB8EEC00AC0EE090ABCEE35
:10543000E00A10EE100A00F57A5020830FE6A0F57E
:10544000F440BB3800EE100AB8EEC00AC0EE090AFC
:10545000BCEEE00A10EE100A30442083FFE5052080
:10546000FBF7A8F953EC182B51EC100B01F0A8FE38
:1054700001F0C2FD80B2608348450ED8A0F56850A7
:10548000BB3800EE100AB8EEC00AC0EE0A0ABCEE45
:10549000E00A10EE100A6083E1E5A0F58E4189393B
:1054A00051450ED8481C00EE100AB8EEC00AC0EEF6
:1054B0000A0ABCEEE00A10EE100A00F57A6060837A
:1054C000CDE5A0F5A841563951450ED8481C00EE4F
:1054D000100AB8EEC00AC0EE0A0ABCEEE00A10EEEE
:1054E000100A00F5FA506083B9E5A0F5C2412339EE
:1054F000B9420DD8481C00EE100AB8EEC00AC0EE42
:10550000090ABCEEE00A10EE100A28446083A6E502
:10551000A0F5DA41EF3941450ED8481C00EE100ADB
:10552000B8EEC00AC0EE290ABCEEE00A10EE100A7E
:1055300000F57A50608392E5A0F5F440B93800EEAA
:10554000100AB8EEC00AC0EE290ABCEEE00A10EE5E
:10555000100A3044608382E50620FBF72BF953ECF8
:10556000182B51EC100B01F02BFE01F045FD80B221
:10557000A08344F28471884210D8A0F56850BA38EC
:1055800000EE100AB8EEC00ADFEDB10A80EE201A74
:10559000BCEEC10A10EE100AA08360E5A0F58E41B2
:1055A000853959450ED8481C00EE100AB8EEC00ADD
:1055B000C0EE2A0ABCEEE00A10EE100A00F57A608E
:1055C000A0834CE5A0F5A8414E3959450ED8481C9A
:1055D00000EE100AB8EEC00AC0EE2A0ABCEEE00ADD
:1055E00010EE100A00F5FA50A08338E5A0F5C2418C
:1055F000173959450DD8481C00EE100AB8EEC00AFC
:10560000C0EE2A0ABCEEE00A10EE100A2844A0837D
:1056100025E5A0F5DA41E03959450ED8481C00EEE1
:10562000100AB8EEC00AC0EE2A0ABCEEE00A10EE7C
:10563000100A00F57A50A08311E5A0F5F440A838CF
:1056400000EE100AB8EEC00AC0EE2A0ABCEEE00A6C
:1056500010EE100A3044A08301E50720FBF7AAF8FA
:1056600053EC182B51EC100B01F0AAFD01F0C4FC17
:1056700080B2E08348450ED8A0F56850BB3800EEF4
:10568000100AB8EEC00AC0EE0A0ABCEEE00A10EE3C
:10569000100AE083E3E4A0F58E41893951450ED824
:1056A000481C00EE100AB8EEC00AC0EE0A0ABCEEB2
:1056B000E00A10EE100A00F57A60E083CFE4A0F56E
:1056C000A8415639B9420ED8481C00EE100AB8EE6F
:1056D000C00AC0EE090ABCEEE00A10EE100A00F59E
:1056E000FA50E083BBE4A0F5C2412239B9420DD89B
:1056F000481C00EE100AB8EEC00AC0EE090ABCEE63
:10570000E00A10EE100A2844E083A8E4A0F5DA418C
:10571000EE3941450ED8481C00EE100AB8EEC00A1A
:10572000C0EE290ABCEEE00A10EE100A00F57A502D
:10573000E08394E4A0F5F440B83800EE100AB8EE27
:10574000C00AC0EE290ABCEEE00A10EE100A30448E
:10575000E08384E40020FBF72DF853EC182B51EC88
:10576000100B01F02DFD01F047FC80B2208448456C
:105770000ED8A0F56850BB3800EE100AB8EEC00A8B
:10578000C0EE0A0ABCEEE00A10EE100A208466E4BD
:10579000A0F58E418939B9420ED8481C00EE100A96
:1057A000B8EEC00AC0EE090ABCEEE00A10EE100A1C
:1057B00000F57A60208452E4A0F5A8415539B94239
:1057C0000ED8481C00EE100AB8EEC00AC0EE090A56
:1057D000BCEEE00A10EE100A00F5FA5020843EE418
:1057E000A0F5C2412139B9420DD8481C00EE100A7B
:1057F000B8EEC00AC0EE090ABCEEE00A10EE100ACC
:10580000284420842BE4A0F5DA41ED39B9420ED8C2
:10581000481C00EE100AB8EEC00AC0EE090ABCEE41
:10582000E00A10EE100A00F57A50208417E4A0F583
:10583000F440B83800EE100AB8EEC00AC0EE090A0B
:10584000BCEEE00A10EE100A3044208407E40000A9
:105850003789513FDFED0A0A20EE200ADFED090A01
:1058600020EE200ADFED080A80EE201ABCEEC10A05
:1058700010EE100A80B20549086000F009B8000077
:105880000000C8420000804500404E452001002035
:105890002DE9F05F4FF6FF7909EA8000C0F30D05AE
:1058A0004FF40058164EC6F81880B714B7610A2096
:1058B00000F080FA7804B0610A2000F07BFA00243E
:1058C0004FF4006A4FF0805BB761280402D5C6F838
:1058D00018A002E04FF00060B0610A2000F06AFA00
:1058E000C6F818B00A2000F065FA09EA4505641CFC
:1058F000E4B2102CE8D3C6F81880BDE8F09F000091
:10590000000C0240DFED090A20EE200ADFED080A54
:1059100020EE200ADFED070A80EE201ABCEEC10A55
:1059200010EE100A80B200F007B800000000C84274
:105930000000804500404E452DE9F05F4FF6FF7BAB
:105940000BEA8000C0F30D054FF48077DFF85CA010
:10595000CAF818704FF40079154EC6F818900A204E
:1059600000F028FA4FF08078CAF818800A2000F07A
:1059700021FA0024C6F81890280401D5B76101E087
:10598000C6F818800A2000F015FA4FF00070B061D8
:105990000A2000F00FFA0BEA4505641CE4B2102C53
:1059A000E8D3CAF81870BDE8F09F0000000002407C
:1059B0000008024010B50446022221492046FAF7A9
:1059C00089FD38B31E4903222F392046FAF782FD9C
:1059D00020B31B4903222B392046FAF77BFD08B37D
:1059E0001749032227392046FAF774FDF0B114490C
:1059F000032223392046FAF76DFDD8B1104903225E
:105A00001F392046FAF766FD002817D1BDE810407F
:105A100000F0A6B9BDE8104000F038B8BDE810406D
:105A200000F0BAB8BDE8104000F018B9BDE8104069
:105A300000F05AB8BDE8104000F03CB910BD0000BD
:105A4000E17900080EB50C490D2001F13202CDE9D3
:105A5000002101F11703029008A232210A48FAF747
:105A6000A3FC0948FAF717FD03B0C1B206485DF878
:105A700004EB00F0F9BA0000AF7900082573257334
:105A800025732563000000003C0700200348012126
:105A900041700278062A00D001707047A0070020EC
:105AA0000EB50C490D2001F10B02CDE9002101F1E9
:105AB0001703029008A232210A48FAF775FC094838
:105AC000FAF7E9FC03B0C1B206485DF804EB00F058
:105AD000CBBA0000AF7900082573257325732563C1
:105AE000000000003C0700203EB500240094019413
:105AF000029415480A22816800780144684600F043
:105B00004FFB01216846425C303A092A01D84254D1
:105B100000E04454491CC9B20729F4D9401C00F0E4
:105B20006DFF9DF800002D2801D1B1EE400A074815
:105B30000178062901D005210170DFED050A20EE6C
:105B4000200A80ED010A3EBD38010020A007002098
:105B500000007A440EB50B490D20CA1CCDE9002186
:105B600001F11703029008A232210A48FAF71CFC3F
:105B70000848FAF790FC03B0C1B206485DF804EBA0
:105B800000F072BAAF790008257325732573256379
:105B9000000000003C0700201CB500240094019484
:105BA00012490878401CC0B2087089680522014477
:105BB000684600F0F5FA0E4968460522491CFAF7D6
:105BC00089FC0C4950B18C700878012805D188787F
:105BD000002802D1012000F00FF81CBD01208870C0
:105BE00008780628F0D002200870EDE73801002080
:105BF000CB790008A00700201FB513490D23CA1D4B
:105C000000280BD001AC01F11C000BC40092431F13
:105C10000EA232211048FAF7C7FB0BE00A4801AC8C
:105C200023300BC40092A0F10C0308A232210A48D1
:105C3000FAF7BAFB0848FAF72EFC04B0C1B2BDE887
:105C40001040054800F010BAAF790008257325739D
:105C500025732573256300003C0700207047002052
:105C600000F04AB8012000F047B800000EB50C491A
:105C70000D2001F10F02CDE9002101F1170302907F
:105C800008A232210A48FAF78FFB0948FAF703FC09
:105C900003B0C1B206485DF804EB00F0E5B90000BE
:105CA000AF79000825732573257325630000000074
:105CB0003C0700201CB50024009401940B4908788F
:105CC000401CC0B20870896805220144684600F093
:105CD00067FA074968460522491CFAF7FBFB0549A4
:105CE00008B1CC701CBD0120C8701CBD380100205B
:105CF000CB790008A00700201FB514490D2301F13E
:105D0000130200280BD001AC01F11C000BC400925F
:105D1000431F0FA232211148FAF746FB0BE00B4854
:105D200001AC23300BC40092A0F10C0308A2322175
:105D30000A48FAF739FB0948FAF7ADFB04B0C1B2DB
:105D4000BDE81040054800F08FB90000AF790008A9
:105D50002573257325732573256300003C070020F8
:105D6000094801780022022906D003780121032B7B
:105D700006D0C27001707047C27003210170704775
:105D8000C170042101707047A00700204FF400513A
:105D900005488161C903816180150449886104490E
:105DA0004004886170470000000C0240000002407F
:105DB0000008024000E000BF401E411CFBD17047BC
:105DC00082B0CDE9000121F0004001909DED000B73
:105DD00002B051EC100B70472DE9F0472DED028B0E
:105DE0002B4C207801284ED104F11402294B206954
:105DF000118823F81010E36801EB0308C4F80C8045
:105E0000244B5188143B23F81010A3681944A16057
:105E1000204B9288283B23F8102063681A44626064
:105E2000401C2061002509282CDD25610A26B2FBD3
:105E3000F6F0194F38806560B1FBF6F040F6E441AA
:105E4000DFF85890484309EB103001F06AF99FEDF4
:105E5000148B53EC182B00F047FF01F0CDF878803D
:105E6000A560B8FBF6F040F6E441484309EB10307A
:105E700001F057F953EC182B00F036FF01F0BCF895
:105E8000B882E5602570BDEC028BBDE8F0870000AC
:105E90003C000020C4010020AC00002024FAFFFFD9
:105EA000CBA145B6F3FDB43FF0B5344D3449354A86
:105EB00028784FF0010406064FF0000303D5E605ED
:105EC0008E61D37102E080268E61D47147064FF453
:105ED000807603D536048E61937101E08E619471F2
:105EE00087064FF4007603D536048E61537101E0C6
:105EF0008E615471C7064FF4806603D536048E61F7
:105F0000137101E08E61147107074FF4006603D529
:105F100036048E61D37001E08E61D47047074FF470
:105F2000805603D536048E61937001E08E619470C3
:105F300087074FF4005603D536048E61537001E095
:105F40008E615470C6074FF4804003D0000488610E
:105F5000137001E0886114706878C10704D00A49A1
:105F60000B6000F0FE0068706878810705D5074A6D
:105F70000221117000F0FD006870F0BDA800002043
:105F8000001002401801002020000020A00700207F
:105F900038B5002100910E4CA060042121700D49FC
:105FA000497800290BD0011D0322684600F0F8F85B
:105FB0002078C01C20706846FFF7FCFC38BD011D2E
:105FC0000222684600F0ECF82078801C2070F2E78E
:105FD00038010020A0070020084900220A708860CC
:105FE0000748C86007480861074848610748886152
:105FF0000748C8610748086270470000A0070020F2
:10600000455A0008555B0008F95B0008A15A0008D2
:106010006D5C0008F95C0008F8B5104D2868C0F305
:10602000001000260E4C002808D0286800906868F0
:10603000009021790B48FFF7ABFF66602868C0F33A
:106040004010002809D06068322800DD6660696869
:10605000044A60681154401C6060F8BD0044004070
:10606000380100206E0700200A4602498B6801466D
:1060700001481847A00700200044004010B5174809
:106080000178062928D0164C2168012924D10178ED
:1060900079B1017801290FD0017802290FD0017858
:1060A00003290FD0017804290FD0007805280FD0DC
:1060B00010E0FFF7C7FC0DE0FFF74CFD0AE0FFF72B
:1060C000CEFD07E0FFF7CEFD04E0FFF7E9FC01E0BD
:1060D000FEF73EFF0020206010BD0000A00700205A
:1060E000800000202A4C00262670FAF767FEFDF794
:1060F000CFFCFCF77DF8FCF72FF8FCF707FAFCF76C
:10610000F1FAFCF70BFCFBF75FFFFCF795F9FCF7E6
:106110009DFCFCF7ADF9FCF71DFBFCF775FBFCF7EC
:1061200059FAFCF719FA1B48016841F001010160B6
:10613000C16841F00101C160416C41F4004141641A
:10614000154D28680128FCD1207840B1012811D0D4
:10615000022813D00328F4D100F0C8FBF1E70F495F
:106160004FF480008861FDF72DF92E602078401CE7
:106170002070E6E7022020702E60E2E700F09EFB30
:106180004020A0612E602078401C2070D9E70000DC
:1061900000000020000400408800002000100240A1
:1061A00003E011F8013B00F8013B521E92B2F8D215
:1061B0007047000010B51D4C206806280CD2DFE89F
:1061C00000F0030C151E283100220421012000F0EC
:1061D000A9FC2068401C206010BD00220521012080
:1061E00000F0A0FC2068401C206010BD00220621A9
:1061F000012000F097FC2068401C206010BD4AF68A
:106200005522FF21022000F08DFC2068401C2060F8
:1062100010BD0122F221022000F084FC2068401C05
:10622000206010BD0620206010BD0000200000206E
:1062300070B52DED108BAD4D9FEDADBB9FEDAECB91
:106240009FEDAFEB9FEDB0FBB14E9FEDB2DB9FED4D
:10625000B3AB286801280AD09FEDB29B02287CD0FE
:10626000032801D101202860BDEC108B70BD00F027
:10627000E3FAAE4C207A00F054FF41EC180BB0EE7C
:106280004B1AF0EE6B1AB0EE4C0AF0EE6C0AFDF70A
:1062900073FFB0EE409AF0EE609AE07900F041FFB3
:1062A00053EC192B00F08CFF53EC182B00F060FC22
:1062B00053EC1A2B00F018FD41EC180BA07900F0FC
:1062C00030FF41EC190BB0EE4B1AF0EE6B1AB0EE4A
:1062D0004C0AF0EE6C0AFDF74FFFB0EE40AAF0EE6C
:1062E00060AA607900F01DFF53EC1A2B00F068FFE4
:1062F00041EC1A0BB0EE4E1AF0EE6E1AB0EE4C0AEC
:10630000F0EE6C0AFDF738FFB0EE40BAF0EE60BA7E
:10631000207900F006FF53EC1B2B00F051FF41ECFD
:106320001B0BB0EE4F1AF0EE6F1AB0EE4C0AF0EE07
:106330006C0AFDF721FFB0EE40CAF0EE60CAE078CB
:1063400000F0EFFE53EC1C2B00F03AFF53EC1B2B3C
:1063500000F00EFC53EC1A2B00E027E000F008FCE4
:1063600053EC192B00F004FC53EC182B00F000FC4C
:1063700041EC100B85ED020B53EC1D2B51EC100B77
:1063800001F01CF801D285ED02DB9FED690B53ECA7
:10639000102B95ED020B51EC100B00F011FF00F0EB
:1063A0002BFE70812868401C28605DE700F049FAE8
:1063B0005E4C2434207A00F0B4FEB0EE4BDAF0EEFE
:1063C0006BDA41EC180BB0EE4D1AF0EE6D1AB0EE30
:1063D0004C0AF0EE6C0AFDF7CFFEB0EE40BAF0EEDC
:1063E00060BAE07900F09DFE53EC1B2B00F0E8FE54
:1063F00053EC182B00F0BCFB53EC1A2B00F074FC90
:1064000041EC180BA07900F08CFE41EC1B0BB0EEB8
:106410004D1AF0EE6D1AB0EE4C0AF0EE6C0AFDF774
:10642000ABFEB0EE40DAF0EE60DA607900F079FEB3
:1064300053EC1D2B00F0C4FE41EC1D0BB0EE4E1AC8
:10644000F0EE6E1AB0EE4C0AF0EE6C0AFDF794FE18
:10645000B0EE40EAF0EE60EA207900F062FE53EC24
:106460001E2B00F0ADFE41EC1E0BB0EE4F1AF0EE0D
:106470006F1AB0EE4C0AF0EE6C0AFDF77DFEB0EE3E
:1064800040CAF0EE60CAE07800F04BFE53EC1C2BE3
:1064900000F096FE53EC1E2B00F06AFB53EC1D2B14
:1064A00000F066FB53EC1B2B00F062FB53EC182B47
:1064B00000F05EFB41EC100B85ED040B53EC192B47
:1064C00051EC100B00F07AFF01D285ED049B95EDA5
:1064D000040B53EC1A2B51EC100B00F071FE00F082
:1064E0008BFDB0812868401C2860BDE64801002073
:1064F00000000000000020400000000000000040FC
:1065000000000000000030400000000000003840A3
:10651000AC00002000000000007884400000000073
:1065200000408F400000000000405040D80700208D
:106530000000000000005940F8B5274C2068C0F367
:106540000010264D0026264B002835D020680090EC
:1065500060680090002029462A784978012A01D1F4
:10656000032902D0022A0AD00BE059681D4A491CAF
:1065700002E02F5C1754401C8842FADB1BE0032921
:1065800002D0032A0BD016E0164A59682432491C5F
:1065900002E02F5C1754401C8842FADB0BE0032911
:1065A00009D1104A59684832491C02E02F5C17543F
:1065B000401C8842FADB5E602068C0F3401000286F
:1065C00008D05868322800DD5E6061685868295438
:1065D000401C5860F8BD00000014014088060020EF
:1065E00048010020D807002010B512480078032881
:1065F0000DD3114B40F2FF34194698880F4A0968B1
:10660000A04205D3002098800860EE20506010BDA5
:1066100052680B4C2270441C9C800A540948016843
:1066200021F00101016000214162016841F0010196
:10663000016010BD00000020C80600200048004096
:106640009000002000140040074A02F588600260B4
:1066500000218180C1800172C2604FF48062028299
:1066600041820248FBF77FBB8802002000480040BF
:1066700070B5084D084B074CDB780C3419510321D9
:106680002846FBF7A3F82846BDE870400321FBF736
:1066900089B80000006002408F79000870B5094891
:1066A0006FF001010161016821F001010160064CF8
:1066B000A088E0800025A58001202072FCF708FB5F
:1066C000257270BD00140040C80600200448C1684F
:1066D00041F00101C160016841F0010101607047B2
:1066E000001400402DE9F041FCF786FE3A4D3B4C8A
:1066F0000A2629780023042925D2DFE801F02402A4
:106700002649A868374A90FBF6FC354F106827F8F1
:1067100010C0401C1060092800DD13600020324AC0
:1067200037F810C0D2F80080C444C2F800C0401C42
:106730000A28F5DB1068B0FBF6F08E1D24F8160071
:106740001360491C2970BDE8F081A868284A90FBB5
:10675000F6FC264F106827F810C0401C106009286E
:1067600000DD13600020234A37F810C0D2F8008003
:10677000C444C2F800C0401C0A28F5DB1068B0FB16
:10678000F6F08E1D24F816001360491C2970DAE714
:10679000A8681A4A90FBF6FC174F106827F810C03B
:1067A000401C1060092800DD13600020144A37F8EF
:1067B00010C0D2F80080C444C2F800C0401C0A28AF
:1067C000F5DB1068891DB0FBF6F024F811001360AA
:1067D00001202870B7E7000024010020AC00002051
:1067E00060010020300000202400002074010020FF
:1067F00034000020280000208801002038000020FC
:106800002C00002010B50B4C207003206070080A8B
:10681000A070E170100A2071062162712046FCF719
:10682000ECF9A071000A0821E0712046BDE8104093
:1068300000F062B9C4070020032204210120FFF701
:10684000E1BF03223C210220FFF7DCBF00B52DEDA4
:10685000048B83B041EC190B00F0F2FD41EC180BF6
:1068600018EE100A18EE901A8DED008B002818BF54
:106870000120084320F00040C0F17F6000F1E040BB
:10688000C00F14D019EE101A19EE900A8DED009B6E
:10689000002918BF0121084320F00040C0F17F60AB
:1068A00000F1E040C00F04BF0120F9F7D2FE51EC27
:1068B000180B03B0BDEC048B00BD000010B5FBF756
:1068C00059FBFAF753F8FDF781FBFFF75FFAFFF783
:1068D000FDFEFFF7B9FEFEF741FB0348FFF77CFB27
:1068E000BDE81040FFF7E0BACD6A000870B52DEDA5
:1068F000028BF3EE098A3C4C9FED3C8A3C4D20888C
:106900003C4E00EE100AF8EE400A80EE880AD5ED03
:10691000040AB4EE600AF1EE10FA13D000EE100A89
:10692000F8EE400A80EE880A85ED040A10EE100A9F
:10693000B04201DDC5ED048AFFF728FA95ED040A9F
:10694000FEF788FF608800EE100AB8EE400AC0EE3D
:10695000080A95ED050AF4EE400AF1EE10FA13D09C
:1069600000EE100AF8EE400A80EE880A85ED050A6E
:1069700010EE100AB04201DDC5ED058AFFF706FAF8
:1069800095ED050AFEF7BEFF287AFEF721FBA86801
:10699000401CA860072801DD0020A860FFF7A2FEC8
:1069A000FFF76CFBFFF718FAFFF77EFA124E30780C
:1069B00000F00400E860FDF715FB6880C1437170CA
:1069C0006FEA10203070E96800F00400884208D0B7
:1069D000A088401C80B2A0804FF6DC71884200D9AC
:1069E000A180BDEC028B70BDDE00002000007A4467
:1069F000000000200000C841AA0000200178174ACA
:106A000040F635435143427812FB03F201EB421149
:106A1000827840F2712312FB03F201EB0212C1787B
:106A200001EB4103C3EBC11102EBC102017901EBA0
:106A3000C10303EB011102EB81024179807901EB83
:106A4000810102EB4101084400EE100A9FED041A97
:106A5000F8EEC00A80EE810A7047000040420F0045
:106A60000050C34730B5164800F10C0151E8002F23
:106A700042F0100241E80023002BF7D11049114DDC
:106A8000091D114C0F4BA2790833D15000F11401AC
:106A900051E8002F42F0800241E80023002BF7D19B
:106AA000A1796958A27941F01001A9500C3050E841
:106AB000001F41F0200140E80012002AF7D130BD4C
:106AC0000044004000600240D979000870B5084DCC
:106AD000084B074C9B790C34195106212846FAF7CC
:106AE00075FE2846BDE870400621FAF75BBE00003F
:106AF000006002408F79000870B5084D084B074CC4
:106B00009B790C3418510A4606212846FAF75EFE96
:106B10002846BDE870400621FAF744BE00640240F2
:106B20008F79000810B50B4C2070062060700B0A9E
:106B3000A370E170110A2171627101462046FCF7D1
:106B40005CF8A071000A0821E0712046BDE8104001
:106B5000FFF7D2BFC407002081F00041704780F0EA
:106B60000040704721F00041704720F0004070471E
:106B700010B591EA030F48BF83F0004300F134855C
:106B8000841A71EB030C05D2121943EB0C03001BA2
:106B900061EB0C01DFF824E14FEA1154A4EB135C24
:106BA0001EEA430F18BF9EEA445F73D023EA0E0328
:106BB000DCF1200E21EA045143F4801332D322FA8F
:106BC0000CFE10EB0E0023FA0CFE41EB0E01CCF193
:106BD000200E03FA0EFE10EB0E0051F10001B1F58C
:106BE000801FCCF1200E32D201EB045112FA0EF2CA
:106BF000BDE8104058BF7047401C38BF5FEA4202F2
:106C000018BF7047002814BF20F0010041F10001B7
:106C10004FEA410313F5001F38BF7047A1F1C0418F
:106C200000F0C6BB012A43EB0302ACF1200CDCF1FF
:106C30001F0E32BF4FF0000E23FA0CF310EB0300CF
:106C400041EB0451B4EB115FD0D0A1EB045101F53D
:106C5000801149085FEA300001EB04510ED350F176
:106C6000000038BF12FA0EFE08D1BDE81040C9E797
:106C7000401C38BF5FEA4202CAD1C3E7BDE81040FA
:106C80004FEA410313F5001F38BF7047A1F1C0411F
:106C900000F08EBB9EEA445F08D011EA5E0FBDE8AB
:106CA000104004BF01F0004100207047BDE81040D3
:106CB00070B500F02FFB00BF64FBBE3E0000E0FF9C
:106CC00002494FF0000000F0D8BD00BF0000F87F7F
:106CD000491058BFC1F140415B1058BFC3F1404358
:106CE0008B42EFF3008070472DE9C04130B4DFF8EC
:106CF000A0C23CEA111418BF3CEA131400F0EC8067
:106D000081EA03051CEA111444EAD57418BF1CEA91
:106D1000131500F0C780A4EB05044FF0004545EAC9
:106D2000C12145EAC32341EA505143EA525304F1D9
:106D30007F74994204F500344FEAC0204FEAC22222
:106D400008BF904200F09C804FEA13650FF2401696
:106D5000765D4FEA134506FB05F7C7F1807706FB22
:106D600007F74FEAD737A7FB03687642C8F58038A4
:106D7000A7FB06CE38BFA8F1010807FB08E64FF0D5
:106D8000000EA6FB028CE6FB03CEDCF1000CCEF17C
:106D9000004E38BFAEF1010EA6FB0C584FF00007B5
:106DA0004FF00005E6FB0E87A1FB08C6A0FB07CE4F
:106DB00016EB0E0645F10005E1FB076515F1E04E07
:106DC0007EBFA4F580345FEA46066D4116F1800768
:106DD00045F100054FEA17274FEA066647EA0567BF
:106DE000A6F1DE46B6F1805F4FEA15251FD9384679
:106DF00024F0010C05EBC471BCF1FE6F01EB0C112A
:106E000002D8F0BCBDE8008124425CBF01F5801EC1
:106E10009EEAC47F02D4F0BCBDE80081244238D48D
:106E2000F0BCA1F1C041BDE8004100F0C1BA4FEA99
:106E3000D22242EA43524FEAD323A7FB02864FEA0B
:106E4000D02040EA415007FB03661EEA0E0F4FEACE
:106E5000D12105FB026658BFA6EB0056B6EB0056E3
:106E60004FEA520E4EEAC37E18EB0E0E56EB530E4F
:106E7000BDD518EB02085E417F1C55F10005B6E751
:106E80004FF480154FF000074FF000064FF0000858
:106E9000ADE7F0BC4FF0000001F1C04101F000414E
:106EA000BDE8008111EA0C1F0CEA131500D00CE0BC
:106EB00013EA0C1F00F025804FF00000F0BC81EABF
:106EC000030101F00041BDE80081F0BCBDE80041D4
:106ED00081EA030100F06CBAF0BCBDE8004170B576
:106EE00000F018FA097EFC3E00F007B881EA0301C1
:106EF0004FF0000001F00041704781EA030100F00B
:106F000057BAF0BCBDE800414FF00000214970477E
:106F1000FFFDFBF9F7F5F4F2F0EEEDEBE9E8E6E45E
:106F2000E3E1E0DEDDDBDAD8D7D5D4D3D1D0CFCDE5
:106F3000CCCBCAC8C7C6C5C4C2C1C0BFBEBDBCBB1E
:106F4000BAB9B8B7B6B5B4B3B2B1B0AFAEADACAB19
:106F5000AAA9A8A8A7A6A5A4A3A3A2A1A09F9F9EF3
:106F60009D9C9C9B9A9999989797969595949393A5
:106F7000929191908F8F8E8E8D8C8C8B8B8A89893C
:106F800088888787868585848483838282818180BF
:106F90000000FF070000F87F4FEA41034FEA535318
:106FA000A3F58063D3F11E03C8BFD3F1210C0CDD20
:106FB0004FF0004242EAC12242EA505232FA03FC48
:106FC0008CEAE17CACEBE1707047102BC4BF002071
:106FD000704703F5787CBCF1FF3F04D06FF00042AE
:106FE00082EA2100704770B500F094F9499224803C
:106FF00000207047F2E700004FEA1153A3F58063C9
:10700000D3F11E03A8BFD3F1200C08DB4FF00042E0
:1070100042EAC12252EA505232FA03F07047094262
:107020000BD4102BC4BF0020704703F5787CBCF153
:10703000FF3F05D04FF0FF3070474FF00000704722
:1070400070B500F067F900BF4992248000207047B6
:10705000F0E710F0004248BF4042B0FA80F310FA67
:1070600003F10AD0C3F11D0303F580634FEA4150D9
:1070700002EB035202EBD12170474FF00000704742
:107080007FEAE17202D1101A62EB0101B1FA81F3D9
:107090000B3B24D3994012D1B0FA80F310FA03F1DC
:1070A00008BF7047C3F11D0303F5406303EBC22320
:1070B0004FEAD1224FEA415002EB03517047C3F12E
:1070C000200C20FA0CFC9840C3F1320303F5406316
:1070D00003EBC22341EA0C0101EB0351704710B5E9
:1070E000C3F1320CC3F10004C4F1200E0CF5406C66
:1070F0000CEBC22201FA0EFC21FA04F100FA0EF3A5
:10710000E040BDE8104040EA0C0001EB025138BFFE
:107110007047401C41F100015B0008BF20F00100F6
:107120007047B0FA80F310FA03F10AD0C3F11D03DF
:1071300003F580634FEA41504FEA035202EBD1213D
:1071400070474FF00000704751EA030C17D41CF54C
:10715000801F58BFBCF5801F00F10680994218BF00
:10716000704708BF9042704707D711F5801F58BF7E
:1071700013F5801F19D499427047894270471CF556
:10718000801F08D5BCF5801FF7D58B4218BF70470C
:1071900008BF824270474FF4001C1CEB410F38BF00
:1071A0001CEB430F01D28B42704770B500F0B2F870
:1071B000922449004FF000514FF08053FFF788BDF3
:1071C000DFF848C170B51CEA111E1EBF1CEA13157A
:1071D0009EEA0C0F95EA0C0F00F06F8081EA030421
:1071E00023EA4C134EEAD47E21EA4C1141F480117B
:1071F00043F48013AE44A1FB024CA0FB0365AEF147
:107200007F7E361955EB0C05A1FB034C4CF10003B6
:10721000A0FB021C16EB0C06654153F1000309426A
:1072200018BF46F0010613F4007F0BD14FEA03317B
:107230004FEA0530340341EA155140EA16506FF029
:1072400003020AE04FEAC3214FEAC520F40241EAF3
:10725000555140EA56506FF0020202EB2E4201EB0C
:10726000025585EACE710AD05FEA440C18BF24F0BB
:10727000004450F1000041F1000120EAD47040F2D6
:10728000FE7C624500D270BDA84214BF4FF080441E
:107290004FF04044002E08BF0024BEF1806FA8BF0D
:1072A000A1F1C041BDE8704080F282804FF0000043
:1072B00001F1C04101F0004170479EEA0C0F0CEA59
:1072C000131518BF95EA0C0F06D04FF0000081EAA5
:1072D000030E0EF0004170BD00F01CF88900013E65
:1072E00000F007B800F009B84FEA430C5FEA5C5CB5
:1072F00008D081EA030100F05BB84FEA410C5FEA75
:107300005C5CF6D14FF00000014970470000FF07B8
:107310000000F87F0EF1020E2EF0030E5EF8046BF3
:10732000364205D4012A43EB030515F5001F12D898
:10733000012841EB010C1CF5001F0CD80ED14FEABF
:10734000D17C15F5001F0CEB4C0C0CF1020C08BFA6
:107350004CEBD37C04E04FF0080C01E04FEAD37C07
:107360000CEB4C0526FA05F606F00706B6F1040C00
:1073700006D20EEB860CBDE870404CF0010C604765
:10738000DFE80CF0090B02024FF000414FF0000063
:10739000A1F5002170BD19461046012851EB0104EA
:1073A00018BFD4F5001484BF002001F0004170BD67
:1073B0000808A0F500114FEA3101704753EA010CAB
:1073C00017D41CF5801F58BFBCF5801F00F1068044
:1073D0008B4218BF704708BF8242704707D713F52A
:1073E000801F58BF11F5801F19D48B4270479B42F4
:1073F00070471CF5801F08D5BCF5801FF7D5994252
:1074000018BF704708BF904270474FF4001C1CEB38
:10741000430F38BF1CEB410F01D2994270470FB4A4
:107420000CBC03BCFFF7C1BE91EA030F10B581F09D
:1074300000413FF5A5AB83F0004300F0D5B8000054
:107440002DE9F04101F5801CBCF5001FC0F2A980B8
:107450004FEA115C21EA0C510CF1FD0C41F4801152
:107460005FEA5C0C0CF5C07C01D34000494130A4BC
:10747000890241EA905187028E0E0A0CA45D04FB3A
:1074800004F602FB06F6C6F14046A4FB0662F60DC2
:1074900046EA422606FB06F4A4FB01235242C3F14E
:1074A000404338BF5B1EA6FB02420024E6FB0324D8
:1074B000D20B42EA4446A6FB0623A1FB02E2A3FB51
:1074C00007E4E3FB61426442C2F1404E38BFAEF1D3
:1074D000010EA6FB04234FF00002E6FB0E32A2FBD6
:1074E00003463400E2FB6264A1FB06E6A4FB07E866
:1074F000E4FB61687642C8F1405838BFA8F1010842
:10750000A2FB06E4A3FB08E5E2FB6854A1FB05E649
:10751000A7FB04E8E1FB648618F1200556F100069C
:10752000A809A8F11B08B10908F03F08B8F10A0F33
:1075300040EA86601CD901EB0C51BDE8F08100BF28
:10754000FCF5EEE8E2DDD8D3CFCBC7C3C0BDB9B6FA
:10755000B4B1AEACA9A7A5A3A19F9D9B9A989695FF
:107560009392908F8D8C8B89888786858483828186
:10757000A0FB006800FB01F208EB4208B8EB87288B
:1075800007D5341858EB0104D5D5401C51F1000142
:10759000D1E7341A78EB0104CDD4401E71F100011B
:1075A000C9E75FEA4C0C5FEA9C5C0DD105D34FF054
:1075B000000001F00041BDE8F081BDE8F04170B588
:1075C000FFF7A8FE6DDBFFBEBDE8F0414FF0000005
:1075D000004970470000F87F10B591EA030F48BFDB
:1075E00083F000433FF5CCAA841A71EB030C07D259
:1075F00012198CF0004C43EB0C03001B61EB0C01E7
:10760000DFF8A4E14FEA1154A4EB135C1EEA430F28
:1076100018BF9EEA445F00F0B08023EA6E03524236
:1076200021EA0451C3EB6E0338BF5B1EDCF1200E70
:1076300025D322FA0CFE10EB0E0043FA0CFE41EBB0
:107640000E01CCF1200E03FA0EFE10EB0E0051F1EC
:107650000001CCF1200E29D412FA0EF201EB0451F4
:10766000BDE8104058BF7047401C1CBFB2F1004F2E
:10767000704700280CBF491C20F00100704712EB36
:10768000020E43EB030218BF4FF0010E4EEA420216
:10769000ACF1200CDCF11E0E54D943FA0CFE10EBB9
:1076A0000E0051F1FF31CCF11E0ED5D50EF1010EB9
:1076B00012FA0EFE404141EB010101EB445C5FEA2E
:1076C0005C5C10D910EBDE7001EB045138BFBEF1E9
:1076D000004FBDE8104018BF704700280CBF491C80
:1076E00020F00100704730D24FEAD42C11F5001180
:1076F00024F400641BD0B1FA81F20B3AA41AA41E40
:10770000D2F12003914030FA03F31943904001EB8A
:10771000CC71002C01EB0451BDE81040A8BF7047AC
:1077200001F1C0414FF0000001F000417047B0FA94
:1077300080F310FA03F100D110BDE41A173C48059C
:10774000C90AE4E701EB045110BD491001EB0451F3
:10775000BDE810404FEA300002E04FF000017047F2
:107760004A0008BF0042F8D0B2F5001F28BF70479A
:1077700001F000414FF0000070479EEA445F07D0DF
:1077800011EA5E0FBDE8104004BF002100207047E1
:10779000BDE8104070B5FFF7BDFD00BF40DFF63E0D
:1077A00083F00041104670470000E0FF4FF040704A
:1077B000E1EE100A704700004FEAC1230A1543EAC0
:1077C00050534FEAC02C18BF43F000431BD4A2F221
:1077D0004E02D2F57C7240F34280502AA8BF50225C
:1077E00023FA02F12CFA02F0D2F1200260B403FA7B
:1077F00002F588BF2843C2F1000223FA02F598BFC0
:10780000284360BC704702F57C7212F5826F08BF96
:1078100023F00043D2F12E0221DB1AD0502AA8BF58
:10782000502223FA02F12CFA02F0D2F1200260B4C5
:1078300003FA02F588BF2843C2F1000223FA02F5D9
:1078400098BF284360BC4042C1F1000138BF491EC7
:1078500070479CF0000F08BF93F0004FDED070B56A
:10786000FFF758FD9224498000214FF00000704737
:107870006FEAE17080F0004170470CF00F03092BB4
:1078800008BF082000F059800A2B0BD0082B18BF26
:10789000704708BF1CF0400F0AD04FF000004FF0B7
:1078A000000170471CF0400F18BF4FF000407047B8
:1078B0001CF0100F08D020F0704300F07F4242EA25
:1078C000D3014FEA4370704700F0604021F07F42DF
:1078D00042EA000201F07F4040EA727070474FF0C8
:1078E000FF0C4CF4E06C1CEA11531CBF9CEA030C27
:1078F0009445C2BFDA4201EB02517047002B0DD014
:10790000BCF1000F0FD0002A01F00041A4BF41F0EC
:10791000E04141F07F614FF00000704701F000410D
:107920004FF00000704750EA01334FF09B0C18BF36
:107930004CF0806C7FF4C4A970471CF4801F11D0F8
:107940001CF4E02F03D06FEACC31490070474FF0B0
:107950004050EFF3008222F0704242EA000282F3CC
:10796000008870474FF0000070471028405870881A
:10797000A0B8000000000404040000080000000893
:1079800000020406080A0C102840587088A0B8109D
:107990002840587088A0B8000000000000000001D6
:1079A0000203040607080900000000010203042A7C
:1079B0002A00524C5200574C5200524D4400525A29
:1079C0005300575A530025303123002B30303030CC
:1079D00031002B303030303000102840587088A0F3
:1079E000B8574353523033303031000000000000AC
:1079F000000000000000F03F000000000000F83F21
:107A000000000000000000000000004003B8E23F5A
:107A1000000000000000000006D0CF43EBFD4C3E0C
:107A2000033333333333E33FFFAB6FDBB66DDB3F01
:107A30004D268F515555D53F01411DA96074D13F49
:107A400065DBC9934A86CD3FEF4E454A287ECA3F43
:107A50003E5555555555C53F93BDBE166CC166BFC5
:107A60002CDE25AF6A56113FF16BD2C541BDBBBEBE
:107A7000D0A4BE726937663E00000000000000001E
:107A8000A07A00080000002060010000C401000886
:107A9000BC7A000860010020480D000020020008A8
:107AA0000118037EFFFF320182103324F412AA0D65
:0C7AB0003655AAAA554C093E8C09362414
:040000050800018965
:00000001FF
